:100000000C9438070C9460070C9460070C946007FC
:100010000C9460070C9460070C9460070C946007C4
:100020000C9460070C9464090C94D3320C944B33F9
:100030000C9460070C9460070C9460070C946007A4
:100040000C94410E0C9460070C9460070C946007AC
:100050000C9460070C9460070C9460070C94402A81
:100060000C9460070C94122F0C944D2F0C94600785
:100070000C9460070C9460070C9460070C94600764
:100080000C9460070C9460070C9460070C94600754
:100090000C9460070C9460070C9460070C94600744
:1000A0000C9460070C9460070C946007D01DD71D5A
:1000B000D71DD01DD71DD71DD71DD71DD71DD71DA7
:1000C000D71DD71DD71DD71DD71DD71DD71D451D22
:1000D000D71DD71DD71DD71DD71DA81CD71DD71DB0
:1000E000D71DD71DD71DD71DD71DD71DD71DD71D70
:1000F000D71DD71DD71DD71DD71D511D511D511DF2
:10010000511D511D511D511D511D511DD71DD71D73
:10011000D71DD71DD71DD71DAD1C501D501D501DFF
:10012000501DD71D611D691D711D791D811D891D02
:10013000911D991DA31DAD1DB71DC11DF41CB41C3F
:10014000D71DD71DD71DD71D451DD71DD71DD71DA1
:10015000D71DD71DD71DD71DD71D4F1D4F1D4F1D97
:100160004F1DD71D611D691D711D791D811D891DC3
:10017000911D991DA31DAD1DB71DC11DF41CB41CFF
:10018000D71DD71DD71DD71D451D081E081E081ECB
:10019000081E081E081E081E081E081E081E081E2F
:1001A000081E081E291F291F291F291F291F291F53
:1001B0004F1E591E631E6D1ED31EDD1EEB1EFD1E3F
:1001C0009A1F0A20DB1FE01FE51FEA1FEF1FF41F25
:1001D000F91F0A2004201127262732273B2748270A
:1001E0006E27762799278627892B8C2B7F2B832BAD
:1001F000AD2BAD2BAD2B902B942B982B9E2BA22BA4
:10020000AD2BA82B456E746572206D656E752E2E14
:100210002E00546F67676C6564206D6963726F5060
:10022000504D00546F67676C656420696E76657227
:100230007465642050504D2100546F67676C65648D
:10024000205458206D7574696E672100546F67677C
:100250006C65642074656C656D65747279210050FD
:10026000726F746F636F6C206572726F7220776942
:1002700074682052580054696D656F7574207768F2
:10028000656E20636F6E6E656374696E6720746F50
:1002900020525800507265737320616E79206B652F
:1002A0007920746F2063616E63656C00436F6E6EBE
:1002B000656374696E6720746F2052582C20706FCC
:1002C00077657220757020746865205258202877F1
:1002D0006974682062696E6420706C756720696655
:1002E000206E6F74207573696E6720616C77617919
:1002F000732062696E642900546F67676C656420BF
:1003000027696D6D656469617465206F75747075BA
:10031000742700546F67676C65642027736C61767F
:1003200065206D6F64652700546F67676C65642096
:1003300027616C776179732062696E642700546F5E
:1003400067676C65642050504D206368616E6E6510
:100350006C206C696D697400536574205253534965
:1003600020696E6A656374696F6E206368616E6E82
:10037000656C2028303D3D64697361626C652900BD
:100380005365742050504D206D696E696D756D20F8
:1003900073796E630053657420626561636F6E20CC
:1003A000696E74657276616C005365742062656174
:1003B000636F6E2064656C617900536574206265BB
:1003C00061636F6E206672657175656E6379206911
:1003D0006E20487A3A20303D64697361626C652C06
:1003E0002050783D504D52206368616E6E656C20E0
:1003F000782C2046783D465253206368616E6E65C6
:100400006C2078005365742050574D2073746F70C2
:100410002064656C61792028302064697361626CA6
:1004200065642C20312D323535203D3D20302E3174
:1004300073202D2035306D696E290053657420506E
:10044000504D2073746F702064656C617920283082
:100450002064697361626C65642C20312D323535FE
:10046000203D3D20302E3173202D2035306D696EBA
:100470002900536574206661696C73616665206448
:10048000656C61792028302064697361626C6564F1
:100490002C20312D323535203D3D20302E3173203A
:1004A0002D2035306D696E29002A2A2A2A2A2A2A07
:1004B0002A2A2A2A2A2A2A2A2A2A2A2A2A2A2A2A9C
:1004C0002A2A2A2A2A2A0052582041636B6564206E
:1004D0002D2072657665727420737563636573731E
:1004E00066756C21002A2A2A2A2A2A2A2A2A2A2AD6
:1004F0002A2A2A2A2A2A2A2A2A2A2A2A2A2A2A2A5C
:100500002A2A002A2A2A2A2A2A2A2A2A2A2A2A2A75
:100510002A2A2A2A2A2A2A2A2A2A2A2A2A2A2A2A3B
:100520000052582041636B6564202D207570646112
:100530007465207375636365737366756C21002A37
:100540002A2A2A2A2A2A2A2A2A2A2A2A2A2A2A2A0B
:100550002A2A2A2A2A2A2A2A2A2A2A2A0056616C80
:1005600069642063686F69636573206172653A200E
:100570005B315D2D5B31365D20286368616E6E6591
:100580006C20312D31362900536574206F757470DD
:10059000757420666F7220706F727420005B585DF6
:1005A0002061626F7274206368616E676573206199
:1005B0006E64206578697420525820636F6E666996
:1005C00067005B535D2073617665207365747469A1
:1005D0006E677320746F205258005B525D20726505
:1005E000766572742052582073657474696E6773EF
:1005F00020746F2064656661756C74730055736553
:10060000206E756D62657273205B312D445D2074C0
:100610006F206564697420706F727473205B452D60
:10062000515D20666F722073657474696E67730024
:10063000202D20726563656976657220636F6E6632
:100640006967757261746F722C20727820737720DD
:10065000000A0A6F70656E4C52536E672000536536
:10066000742073657269616C206261756472617473
:10067000653A200056616C69642063686F69636540
:10068000733A2031202D20342B34202F2032202D7E
:100690002038202F2033202D20382B34202F2034B9
:1006A000202D203132202F2035202D2031322B34A7
:1006B000202F2036202D20313600536574204368CA
:1006C000616E6E656C20636F6E6669673A200053D9
:1006D00065742044617461726174652028302D3224
:1006E000293A200053657420486F70206368616E5A
:1006F0006E656C7320286D61782032342C20736510
:100700007061726174656420627920636F6D6D61E0
:1007100073292076616C69642076616C756573203D
:10072000312D3235353A2000536574206368616E8F
:100730006E656C2073706163696E67202878313054
:100740006B487A293A200053657420524620706F16
:100750007765722028302D37293A200053657420A0
:100760005246206D61676963202868657829206595
:100770002E672E20307844454144463030443A209C
:1007800000536574206261736520667265717565DA
:100790006E63792028696E20487A293A20005B5AD6
:1007A0005D20656E74657220726563656976657239
:1007B00020636F6E66696775726174696F6E20750C
:1007C00074696C79005B465D20646973706C617953
:1007D0002061637475616C206672657175656E6306
:1007E0006965732075736564005B525D2063616C9D
:1007F00063756C6174652072616E646F6D206B65EA
:100800007920616E6420686F70206C697374005B7E
:10081000495D207265696E697469616C697A6520E9
:1008200073657474696E677320746F20736B65747D
:1008300063682064656661756C7473005B585D2045
:10084000726576657274206368616E676573206196
:100850006E642065786974206D656E75005B535D0C
:1008600020736176652073657474696E6773207494
:100870006F20454550524F4D20616E642065786968
:1008800074206D656E7500557365206E756D6265BB
:100890007273205B302D395D20746F20656469743C
:1008A00020706172616D657465727300202D205334
:1008B000797374656D20636F6E66696775726174B4
:1008C000696F6E000A0A6F70656E4C52536E672036
:1008D000005129204F7574707574206265666F72BF
:1008E00065206C696E6B20283D465329203A200014
:1008F000502920536C617665206D6F6465202865F2
:1009000078706572696D656E74616C293A20004F6C
:10091000292054696D65642042494E442061742049
:100920007374617274757020203A20004E29205033
:10093000504D206F7574707574206C696D697465A5
:100940006420202020203A200044495341424C4555
:1009500044004D292050504D205253534920746F6C
:10096000206368616E6E656C202020203A20004C68
:10097000292050504D206D696E696D756D20737919
:100980006E63202875732920203A20004449534182
:10099000424C4544004B29204661696C7361666591
:1009A00020626561636F6E20696E74762E20283137
:1009B0002D32353573293A20004A29204661696C69
:1009C0007361666520626561636F6E2064656C614A
:1009D000792028302D323535203D3E2031307320AE
:1009E0002D203135306D696E293A20004929204685
:1009F00061696C7361666520626561636F6E206614
:100A000072712E203A200048292050574D207374CF
:100A10006F702064656C6179202020202020203AAE
:100A2000200047292050504D2073746F702064655A
:100A30006C6179202020202020203A2000462920A7
:100A40004661696C736166652064656C617920201C
:100A500020202020203A200050574D206368616EEE
:100A60006E656C200066756E6374696F6E3A200067
:100A70002920706F72742000506F776572546F7701
:100A8000657200445446205548462033322D626931
:100A9000742031306368004F70656E4C52536E673E
:100AA0005258206D696E6920342F36636800466C99
:100AB0007974726F6E2F4F72616E67655258205550
:100AC00048462038636800525820747970653A208F
:100AD0000044697361626C656400487A00203D3DA2
:100AE000200043616C63756C6174656420706163A0
:100AF0006B657420696E74657276616C3A20004291
:100B000029204D6963726F202868616C6629205026
:100B1000504D202020203A00412920496E766572F0
:100B20007465642050504D20696E20202020203AAA
:100B3000003029204D7574652062757A7A657220BF
:100B4000286D6F73746C79293A00392920536572C6
:100B500069616C2062617564726174653A00736DDD
:100B6000617274506F7274004672536B79005472E4
:100B7000616E73706172656E740044697361626C5A
:100B800065640038292054656C656D657472793A26
:100B900020202020202020003729204368616E6E0D
:100BA000656C20636F6E6669673A202000362920E5
:100BB00044617461726174652028302D32293A20B5
:100BC000202000352920486F70206368616E6E65B3
:100BD0006C733A2020202020003429204368616E65
:100BE0006E656C2073706163696E673A2020003314
:100BF0002920524620706F7765722028302D3729C2
:100C00003A202020003229205246206D6167696316
:100C10003A2020202020202020200031292042615D
:100C20007365206672657175656E63793A20202060
:100C30000000000000240027002A002D00300000E2
:100C4000000000250028002B002E003100000000CD
:100C5000002300260029002C002F000404040404B3
:100C6000030405020202020403020202020606064F
:100C70000606060404020202040408020110408071
:100C80004010204080408008020401804020100273
:100C9000011080102040400000000200080E0000FB
:100CA000030401000B000000000000000000000031
:100CB0000000000000070605040100080A0B0C0DE7
:100CC00009080B00020202010009040000010202EF
:100CD000000005240010010524010101042402067E
:100CE00005240600010705810310004009040100E6
:100CF000020A000000070502024000000705830207
:100D000040000004030904220341007200640075DE
:100D10000069006E006F0020004C0065006F006EDF
:100D2000006100720064006F0018034100720064EB
:100D300000750069006E006F0020004C004C0043FD
:100D40000012010002000000404123368000010132
:100D5000020001120100020200004041233680001F
:100D6000010102000100C18081C105010902A10148
:100D70000901A100850105091901290315002501B3
:100D800095037501810295017505810305010930FF
:100D9000093109381581257F750895038106C0C082
:100DA00005010906A1018502050719E029E71500DB
:100DB0002501750195088102950175088103950645
:100DC0007508150025650507190029658100C0090A
:100DD0000402000103000000092101010001226555
:100DE000000705840340000100000000000000002F
:100DF0002A2B280000000000000000000000000076
:100E000000000000000000002C9EB4A0A1A2A434A9
:100E1000A6A7A5AE362D3738271E1F202122232452
:100E20002526B333B62EB7B89F8485868788898AEE
:100E30008B8C8D8E8F909192939495969798999A8A
:100E40009B9C9D2F3130A3AD350405060708090A88
:100E50000B0C0D0E0F101112131415161718191A6A
:100E60001B1C1DAFB1B0B5005C2CF5303132B9346C
:100E700011241FBECFEFDAE0DEBFCDBF13E0A0E04C
:100E8000B1E0E8E0FDE602C005900D92A03CB1079C
:100E9000D9F716E0A0ECB3E001C01D92A73EB10760
:100EA000E1F71EE0C0E7DEE004C02297FE010E94E9
:100EB0005F36C836D107C9F70E943A310C948236A2
:100EC0000C940000A0E0B0E0E8E6F7E00C942E36C9
:100ED000EC01A880B980CA80DB80A114B104C104F0
:100EE000D10441F484E2A82E89EDB82E8BE5C82EFA
:100EF00087E0D82EC601B5012DE133EF41E050E087
:100F00000E940B3627EA31E440E050E00E94B735FA
:100F10007B018C01C601B5012DE133EF41E050E0CA
:100F20000E940B36CA01B9012CEE34EF4FEF5FEF90
:100F30000E94B7356E0D7F1D801F911F97FF04C063
:100F40006150704080409048688379838A839B8396
:100F50009B01AC015F77B901CA01CDB7DEB7EAE00A
:100F60000C944A360E946207089581EB92E00E9439
:100F7000620708956093B1027093B2028093B30246
:100F80009093B4020895A0E0B0E0E9ECF7E00C948F
:100F90002736EC012B016A016115710519F0FB017F
:100FA00091838083C114D10449F0C60102978397CD
:100FB00028F020E030E040E050E0DCC0A9908A2D2D
:100FC00090E00E947736892BC9F7FDE2AF1621F435
:100FD000A9903324339405C08BE2A81609F4A99094
:100FE0003324C114D10421F0E0E1CE16D10411F56F
:100FF000F0E3AF1669F48881883711F0883541F441
:10100000A980229682E0382A20E1C22ED12C12C07B
:10101000C114D10479F4E0E3AE1659F199E9E92E4F
:1010200099E9F92E99E9092F99E1192F8AE0C82E3B
:10103000D12C3AC0FAE0CF16D10491F080E1C81665
:10104000D10429F0E8E0CE16D104F9F415C0BFEFC1
:10105000EB2EBFEFFB2EBFEF0B2FBFE01B2F24C0EB
:10106000A9E9EA2EA9E9FA2EA9E90A2FA9E11A2F7E
:101070001BC0F8E0CF2ED12CEFEFEE2EEFEFFE2EBF
:10108000EFEF0E2FEFE11E2F0FC09601442737FD23
:101090004095542F6FEF7FEF8FEF9FEF0E94E93560
:1010A000C901DA017C018D0120E030E040E050E030
:1010B00060E03601882477FC8094982C70EDB72E80
:1010C000BA0CF9E0FB1570F48A2D81548A3118F4BA
:1010D00099ECB92E06C08A2D81568A3148F589EAE5
:1010E000B82EBA0C8B2D90E08C159D050CF56F3F3A
:1010F000E9F0E216F30604071507B8F0CA01B901D2
:10110000A40193010E94B7359B01AC018B2D90E0A7
:10111000A0E0B0E0280F391F4A1F5B1F28173907CE
:101120004A075B0710F061E001C06FEFA990C6CFDE
:101130004114510451F0662311F0219703C031FE90
:1011400004C02297F201D183C08330FE07C05095BE
:101150004095309521953F4F4F4F5F4F67FF0AC035
:1011600082E290E09093E6068093E5062FEF3FEF52
:101170004FEF5FEFB901CA01CDB7DEB7E1E10C94E3
:101180004336FC0188279927E89421912032E9F31E
:10119000293010F02E30C8F32B3241F02D3239F4C3
:1011A000689404C00E941609820F911D219120535A
:1011B0002A30C0F31EF4909581959F4F089540EC1E
:1011C00053E00E94E4080895009731F4DA018D910C
:1011D0009C91009709F40EC0DC01FB013D91219127
:1011E000222319F03217C9F3FACF332331F4DA018D
:1011F0001D921C928827992708951197AF93BF934A
:10120000FB013D912191321771F4332321F488279A
:101210009927119702C01E921196FA01A193B083EB
:101220009F918F910895222369F7EACF7AE0979FE3
:10123000902D879F802D910D112408958091C203D8
:10124000813019F482E08093C2038091C20383301D
:1012500019F484E08093C2030895009721F19C0162
:1012600040E050E068E478EE81E090E00E940B36C8
:10127000C901DA018F3F9105A105B10531F028F0D0
:101280008FEF90E0A0E0B0E008C00097A105B105A5
:1012900021F481E090E0A0E0B0E08093D100809163
:1012A000C000806103C08091C0008F7E8093C00029
:1012B0000895EBE6F0E0808180688083E8E6F0E066
:1012C00080818160808308951F920F920FB60F92E4
:1012D00011242F933F934F935F936F937F938F933B
:1012E0009F93AF93BF93EF93FF931F9902C00E9408
:1012F0001E09FF91EF91BF91AF919F918F917F91C7
:101300006F915F914F913F912F910F900FBE0F9072
:101310001F90189581E008951F93182F0E948A0945
:101320008823E9F02FB781E08093C905F894809174
:101330000008909101088757974709F0A89588E120
:101340008093600010936000112341F080910008A9
:10135000909101088757974709F0A8952FBF1F91D3
:101360000895382F20E080915B0590915C058227DD
:10137000932740E061E270E19C01220F331F97FF49
:1013800004C0C9018627972701C0C9014F5F4830B3
:1013900099F790935C0580935B05089587E38093AC
:1013A000F80380E092ECA1E0B0E08093F903909321
:1013B000FA03A093FB03B093FC0387E0809305043A
:1013C00080EC9AECA9E8B6E38093FD039093FE03CA
:1013D000A093FF03B093000485E0809306048DEE94
:1013E0009EEFADEABEED8093010490930204A093BA
:1013F0000304B0930404A7E0B4E080E090E08630FA
:1014000010F0E0E004C0FC01E657FC4FE081ED93F2
:1014100001968831910599F782E080931F048AE054
:1014200080932004089580EC97EFAAEBB7E38093B4
:10143000C5039093C603A093C703B093C80380E08D
:1014400090E0A0E0B0E58093C9039093CA03A09315
:10145000CB03B093CC03EDECF3E080E081938F5F9E
:101460008031E1F708958436910520F4BC0180E0D5
:1014700090E025C08E3B910550F48A559040BC0108
:1014800080E090E02AE030E040E050E016C0823D8D
:10149000910550F4845B9040BC0180E090E024E62C
:1014A00030E040E050E009C08D5C9040BC0180E03D
:1014B00090E028E532E040E050E00E94B73524E6B5
:1014C00030E040E050E00E94B735089590E08C593C
:1014D0009F4F0E94330A0895DC019896EC91F0E04A
:1014E000E770F070EE57FC4F808108958F929F92C5
:1014F000AF92BF92CF92DF92EF92FF920F931F9322
:101500008C010E946C0AD80197962C9130E043E13F
:1015100050E0249FF001259FF00D349FF00D112421
:10152000EB54FD4F80809180A280B38090E00F96B5
:10153000AA2797FDA095BA2FBC01CD0120E43FE179
:101540004DE750E00E94B735A50194010E94E935AE
:1015500069017A0180ED97E0A0E0B0E0C80ED91EE5
:10156000EA1EFB1ED80198968C91887181F060E08C
:101570007EEE8AEB9BE0A50194010E94E93528519B
:101580003C4F4F4F5F4FC20ED31EE41EF51E87EE39
:1015900093E0A0E0B0E0C80ED91EEA1EFB1EC70112
:1015A000B60128EE33E040E050E00E94E935CA0180
:1015B000B90128EE33E040E050E00E94B7351F91BA
:1015C0000F91FF90EF90DF90CF90BF90AF909F90E2
:1015D0008F9008958F3F910509F010F480E00895F1
:1015E00022E08030920710F481E00895805093400B
:1015F00010F083E0089582E00895CF92DF92FF9289
:101600000F931F93CF93DF93F82FEB016A01182FED
:101610001695E0E088819981D6018C938A819B811F
:1016200011968C9311978C819D8112968C931297B1
:101630008E819F8113968C931397288139814A81DB
:101640005B816C817D818E819F819295990F990F2D
:10165000907C832F8370982B852F8370880F880F41
:10166000982B872F83708295807F982B14969C935C
:1016700085E090E0C80ED91E2896EF5F1E1750F641
:10168000F0FF21C0888199810E94EA0AF82E8A81A0
:101690009B810E94EA0A182F8C819D810E94EA0A90
:1016A000082F8E819F810E94EA0AF294FF0CFF0CA2
:1016B00070ECF7221295107F1F29182B000F000FD6
:1016C000012BD6010C93DF91CF911F910F91FF90C9
:1016D000DF90CF90089523E08032920718F420E045
:1016E00030E026C023E0883E920748F49C012F5149
:1016F000334054E0369527955A95E1F719C027E015
:10170000803D920720F49C012C5D334011C028E0FD
:101710008839920718F02FEF33E00AC09C01285C4B
:10172000374044E0369527954A95E1F72D503C4FD8
:10173000C90108958C30910548F49C0174E0220F92
:10174000331F7A95E1F7285D3C4F17C023E0843FB3
:10175000920720F49C0124523C4F0FC024E08030BB
:10176000920718F020E938E008C09C012657334F53
:1017700064E0220F331F6A95E1F7C90108959C01C7
:101780003695279525753575821B930B9C013695EB
:101790002795369527952373337383739373280F97
:1017A000391FC901E4E096958795EA95E1F7820F24
:1017B000931F8F709F7021E031E0AC01429FC00108
:1017C000439F900D529F900D1124892F08958823D7
:1017D00039F0299800002A9A0000299A00000895FB
:1017E000299800002A980000299A00000895299A53
:1017F000000083B12998000090E0B3E096958795AA
:10180000BA95E1F7817008950F931F93082F5E9AA0
:1018100029985E9810E0802F80780E94E70B000FD7
:101820001F5F1830C1F729981F910F9108958F7786
:101830000E94040C08950F931F93082F10E0802F2F
:1018400080780E94E70B000F1F5F1830C1F72998BE
:101850001F910F9108950F931F93299880E000E046
:10186000182F110F0E94F70B810F0F5F0830C1F77F
:101870001F910F9108950E94170C0E942B0C5E9AE5
:1018800008951F93162F80680E94040C812F0E94D8
:101890001B0C5E9A1F9108951F9310910104182745
:1018A000E8EFF3E0E80FF11D89E767850E94410C3E
:1018B0008DE3612F0E94410C82E4612F0E94410C54
:1018C0001F91089586E20E943B0C08950F931F9389
:1018D0008C018CE1F80164810E94410C8DE1F801DA
:1018E00065810E94410C8EE1F80166810E94410CE5
:1018F00080E2F80167810E94410C81E2F801608575
:101900000E94410C82E2F80161850E94410C83E251
:10191000F80162850E94410C84E2F80163850E940F
:10192000410C85E2F80164850E94410C8AE2F801CD
:1019300065850E94410C8EE6F80166850E94410C87
:101940008FE6F80167850E94410C80E7F801608905
:101950000E94410C81E7F80161890E94410C82E7F5
:10196000F80162890E94410C1F910F910895EF9236
:10197000FF920F931F93CF93DF937B018C01603015
:1019800028E372072CE982072CE1920728F520E86A
:1019900036E948E950E00E94E935E9016897B90164
:1019A00080E090E020E839E647E65FEF0E94B73537
:1019B0006E0D7F1D801F911F32E0660F771F881FFD
:1019C000991F3A95D1F721E732E040E050E00E94BC
:1019D000E935890180E421C020E03DE241E351E0A6
:1019E0000E94E935E9016897B90180E090E020E0C4
:1019F00033ED4EEC5EEF0E94B7356E0D7F1D801FFC
:101A0000911F660F771F881F991F21E732E040E082
:101A100050E00E94E935890180E69E012F71622F16
:101A2000680F85E70E94410C86E7612F0E94410CF8
:101A300087E7602F0E94410CCDB7DEB7E6E00C943B
:101A40004E369F92AF92BF92CF92DF920F93DF9369
:101A5000CF9300D000D0CDB7DEB7982E83E00E94A0
:101A60003B0C8093210484E00E943B0C8093220471
:101A700086E060E00E94410C87E061E00E94410C3A
:101A800089E06FE70E94410C8AE065E00E94410C0A
:101A90008BE065E10E94410C8CE062E10E94410C08
:101AA0008DE06DEF0E94410C8EE060E00E94410CE1
:101AB000992019F084E193E008C080911F0423E18C
:101AC000829FC00111248B549D4F0E94660C80E3BD
:101AD0006CE80E94410C82E36FE00E94410C83E3BA
:101AE00062E40E94410C84E36AE00E94410C85E3B9
:101AF0006AE20E94410C86E36DE20E94410C87E39A
:101B000064ED0E94410C88E360E00E94410C89E38F
:101B100060E00E94410C992049F065E8A62E61EC36
:101B2000B62E61ECC62E6EEDD62E08C0A090010434
:101B3000B0900204C0900304D09004040AE38D2DF9
:101B40009927AA27BB2789839A83AB83BC83802FDD
:101B500069810E94410C802F8B5F69810E94410C3A
:101B6000DC2CCB2CBA2CAA240F5F0E3341F783E474
:101B70006FEF0E94410C84E46FEF0E94410C85E4FA
:101B80006FEF0E94410C86E46FEF0E94410C992098
:101B900019F08DE666E003C08DE6609105040E94B1
:101BA000410C89E760E00E94410C8AE760910604DD
:101BB0000E94410C83E760E00E94410C84E760E0F2
:101BC0000E94410C992029F060EC7AEC89E896E3B8
:101BD00008C06091FD037091FE038091FF03909116
:101BE00000040E94B70C0F900F900F900F90CF91B0
:101BF000DF910F91DF90CF90BF90AF909F900895AD
:101C000087E061E00E94410C8EE764E20E94410C93
:101C100088E063E00E94410C88E060E00E94410C93
:101C200087E065E00E94410C85E062E00E94410C83
:101C300083E00E943B0C8093210484E00E943B0CD3
:101C4000809322040895582F4091C604842F90E079
:101C5000FC01EF70F0709F012F5F3F4F74E095958E
:101C600087957A95E1F72817390751F0EA54FB4F29
:101C70005083842F8F5F8F70407F842B8093C604A6
:101C800008951F920F920FB60F9211241F932F9356
:101C90003F934F935F936F937F938F939F93AF93F4
:101CA000BF93CF93DF93EF93FF93C0918600D091C2
:101CB000870020910805309109058091E704882369
:101CC00009F062C0BE01621B730B2091C903309101
:101CD000CA034091CB035091CC0325FD02C07695F9
:101CE000679589E0653C7807B8F1809147031CE16E
:101CF00056954795379527951A95D1F721153105B2
:101D00004105510521F421E030E040E050E090E051
:101D1000A0E0B0E0281739074A075B07D0F48091AC
:101D200047038F3FB1F020E00EC0E22FF0E0EE0F4E
:101D3000FF1FDF01A851BB4F8D919C91E95DFC4FC6
:101D4000918380832F5F80914703281770F310924F
:101D5000E6041092470318C082E06D3B780760F1FB
:101D600080914703803140F510914703CB010E94D9
:101D70006B0BE12FF0E0EE0FFF1FE851FB4F91835B
:101D800080831F5F10934703D0930905C093080514
:101D9000FF91EF91DF91CF91BF91AF919F918F9183
:101DA0007F916F915F914F913F912F911F910F9074
:101DB0000FBE0F901F9018958FEF80934703E4CFCD
:101DC00083E0809380008AE9809381008091C90339
:101DD00086FD05C0809181008064809381008FEF33
:101DE0009FEF909389008093880080916F008062BC
:101DF00080936F0008956F3018F08695805808958D
:101E000089E0689F802D11240895882319F460E0EB
:101E100071E002C063E071E087E196E00E94FD2E70
:101E20000895A0E0B0E0E7E1FFE00C943036182F11
:101E30000E94962A9B01AC01809155059091560510
:101E4000A0915705B091580569017A01C81AD90ABD
:101E5000EA0AFB0AD701C60189589341A040B04065
:101E600010F0109254052093550530935605409379
:101E70005705509358052091E704822F81508230F6
:101E8000E8F580915405882309F44FC1813011F49D
:101E900082E0BCC1803108F035C1E82FF0E0E851A4
:101EA000FB4F10838F5F80935405803109F0B0C1E0
:101EB000AAEEB4E0213039F41196EC911197E69531
:101EC000E6958C9109C08D919C911197E92FE6952B
:101ED000E695E69596958795E03140F4F0E090E040
:101EE000EE0FFF1FE95DFC4F918380831092E604A3
:101EF000129684E0A83FB807E9F68AC1233009F0BA
:101F000004C180915405882321F41F3009F080C159
:101F10000CC1883130F4E82FF0E0E951FB4F108319
:101F200074C1883109F0EEC0112309F0EBC0C0E0A4
:101F3000D0E00BE010E0DE0163E0AA0FBB1F6A9562
:101F4000E1F7C09FB001C19F700DD09F700D1124AB
:101F5000FB01E851FB4F80812181922F977095956D
:101F60008795FD01EE0FFF1FE95DFC4F9183808394
:101F7000FB01E751FB4F308136953695369521812F
:101F8000422F4295440F407E842F832B2695269521
:101F90002695922F977095958795FD01EE0FFF1F5F
:101FA000E75DFC4F91838083FB01E651FB4F80810D
:101FB00082958695869583704181942F990F990F0C
:101FC000292F282B42954695469543708281817032
:101FD000880F880F382F342B35952795FD01EE0F8C
:101FE000FF1FE55DFC4F31832083FB01E451FB4F74
:101FF000308136952181422F479544274795842F7C
:10200000832B2695922F977095958795FD01EE0F5E
:10201000FF1FE35DFC4F91838083FB01E351FB4F86
:10202000308132953F702181422F4295407F842F2D
:10203000832B22952F70922F977095958795FD0190
:10204000EE0FFF1FE15DFC4F91838083FB01E251A6
:10205000FB4F8081881F8827881F4181942F990F0B
:10206000292F282B441F4427441F82818370880F07
:10207000382F342B35952795FD01EE0FFF1FEF5CB0
:10208000FC4F31832083FB01E051FB4F30813695BB
:1020900036952181422F4295440F440F407C842F76
:1020A000832B26952695922F977095958795AA0F45
:1020B000BB1FFD01ED5CFC4F918380836F507B4F14
:1020C000FB0120812295269527704181342F330F03
:1020D000330F330F832F822B942F92959695977001
:1020E00095958795AB5CBC4F11969C938E932196EA
:1020F000C230D10509F01FCF8091FE0483FD02C0DC
:102100001092E6041092540583C0243009F080C078
:1021100040915405442359F4183AB1F410925C05E7
:1021200010925B0588EA0E94B10981E06FC04130DE
:1021300019F41093590504C0423031F410935A0534
:10214000812F0E94B1095DC060915A05262F30E0B1
:10215000220F331FE42FF0E0C90102968E179F076C
:1021600034F0433268F7EB51FB4F1083E9CF2D5F1A
:102170003F4F40915B0550915C05E217F30749F42E
:10218000912F80E04827592750935C0540935B05C9
:1021900038C0812F90E04817590789F5809159057B
:1021A000813069F5613118F080E180935A05D09053
:1021B0005A0548EEE42E44E0F42E00E010E01BC087
:1021C000F701D081C0E0818190E08C2B9D2B33E022
:1021D000969587953A95E1F70E946B0BF801EE0F03
:1021E000FF1FE95DFC4F918380830F5F1F4F82E0EB
:1021F00090E0E80EF91E0D1518F31092E604109207
:10220000540580915405882319F08F5F80935405FD
:10221000CDB7DEB7E8E00C944C36FF920F931F93D6
:10222000CF93DF93182F092FF62E8EE30E94410CD7
:10223000212F302FC901EC0110E005C08FE7699113
:102240000E94410C1F5F1F15C8F385E064E00E94E7
:10225000410C83E00E943B0C8093210484E00E94A7
:102260003B0C809322040E94962A6093230470936F
:102270002404809325049093260487E069E00E945B
:10228000410C81E08093C203CDB7DEB7E5E00C944A
:102290004F360E940D118091C2038130D9F40E9403
:1022A000962A2091230430912404409125045091D2
:1022B0002604621B730B840B950B605A7648814091
:1022C000904040F4E8CF87E196E067E071E00E943B
:1022D000FD2E08958091C2038130A9F308958DEAFF
:1022E00096E06EE70E94B5300895A0E0B0E0EBE71D
:1022F000F1E10C942F366C018DEA96E06EE70E94B6
:10230000B530760100E010E0C0E0D0E0B0E2BB2ED6
:102310000AC00830110521F49E012095F60120879E
:102320000894E11CF11CF7016081862F8D578230E3
:1023300040F48DEA96E06DE70E94B530F7016081C8
:102340006B258DEA96E00E94B5300115110551F01C
:10235000F70180819E01280F311DC32FDD27C20F99
:10236000D31FD0700F5F1F4F0930110591F6CDB705
:10237000DEB7E9E00C944B36A9E0B0E0E2ECF1E125
:102380000C943636382FE62F8091CB0490E00196DE
:1023900064E270E00E94D635982F8093CB0488E9E0
:1023A000898380E18A83913071F0913028F09230F6
:1023B00099F09330E1F416C085E08B8381EF8C8334
:1023C0002F5F2D8317C09B8381EF8C8384E6489F0A
:1023D000C00111249D830EC084E08B8381EF8C8328
:1023E0003D8308C09B8381EF8C83ED8303C00E94F3
:1023F0006F1104C0CE0101960E9475112996E2E08A
:102400000C9452360F931F93CF93DF93182F092FFD
:102410008DEA96E06EE70E94B530212F302FC9017A
:10242000EC0110E000E288818D57823040F48DEAA3
:1024300096E06DE70E94B5308881802788838DEA19
:1024400096E069910E94B5301F5F193061F78DEAFF
:1024500096E06EE70E94B530DF91CF911F910F910A
:102460000895A9E0B0E0E7E3F2E10C943636382FA6
:102470008091CB04882379F48EEF89833A836B8330
:10248000842F90E0959587958C832D8319861886E7
:102490001F821E822FC04091C604842F90E09C01B1
:1024A0002F70307054E0959587955A95E1F7821713
:1024B000930721F18DEF89831A821B82DE01149626
:1024C00020E008C0EA54FB4F80818D93405F2F5F6E
:1024D000263069F0842F90E0FC0134E0F595E79513
:1024E0003A95E1F78F709070E817F90759F7409324
:1024F000C6042A83CE0101960E9402128091CB0469
:1025000090E0019666E070E00E94D6358093CB049F
:102510002996E2E00C9452369F92AF92BF92CF92EE
:10252000DF92EF92FF920F931F93B82EA62ED42E18
:10253000C22E902E0E94962A7B018C018091B504B8
:102540002091C7043091C8044091C9045091CA0435
:102550008823B1F0D801C701821B930BA40BB50BE4
:10256000815E9E42A040B04020F12C2DDC1408F486
:102570002D2D8B2D6A2D422F292D0E94BC1111C0AB
:10258000D801C701821B930BA40BB50B8153954750
:10259000A040B04070F08B2D6A2D4D2D2C2D0E9447
:1025A0003112E092C704F092C8040093C90410935A
:1025B000CA041F910F91FF90EF90DF90CF90BF90D2
:1025C000AF909F900895E82FF0E0EC53FC4FE18529
:1025D000E03148F4F0E0EE0FFF1FE95DFC4F0190A1
:1025E000F081E02D13C0E03129F0E13129F0E0E085
:1025F000F2E00CC082E001C083E00E94E12B892B55
:1026000019F4ECE0F0E002C0E4EFF3E0CF0108954C
:10261000A0E2B0E0EEE0F3E10C942E368CE00E94F4
:102620003B0C882379F587E196E063E171E00E9435
:10263000FD2E5F9A80E00E94210D0E94000E5F989F
:1026400021C08DEA96E00E947C30482F8091E704FB
:10265000882321F0842F0E94110F14C0809152050D
:10266000E82FF0E031969F012F7130703197809103
:10267000510590E02817390729F0E85DFA4F4083AB
:10268000209352058DEA96E00E944230892BC9F6CC
:102690008091E704882339F40CC087E196E00E941A
:1026A000392C0E94110F87E196E00E94122C892B91
:1026B000A1F78091C203843009F08EC00E94962A4F
:1026C0006093D6047093D7048093D8049093D90470
:1026D000611571058105910561F481E090E0A0E04C
:1026E000B0E08093D6049093D704A093D804B0931D
:1026F000D9048091E2049091E30481609093E30413
:102700008093E20483E08093C2038FE70E94170C5A
:102710000FE115E00E942B0CF80181938F01F5E089
:1027200008321F07B9F740910A0580911F05282F2D
:1027300030E0842F90E08227932786FF40C080E41A
:10274000482740930A05C90188739070C89709F516
:1027500010E014C01F5F80912004E12FF0E084FF9F
:1027600006C0E15EFA4F80810E94230E07C0E15E41
:10277000FA4F8DEA96E060810E94B530212F30E05B
:1027800080911F0590E0877090708217930714F76F
:1027900016C02F733070232B91F480912005809305
:1027A000DA04809121058093DC04809122058093D6
:1027B000DD04809125058093E4041092E504809166
:1027C0005305813019F482E08093530580915305BD
:1027D000833011F4109253050E94962A5B016C011C
:1027E0008091DE049091DF04A091E004B091E104B7
:1027F0000097A105B105C9F086017501E81AF90A2B
:102800000A0B1B0BD801C701885B9B40A040B0405E
:1028100060F00E94620C8093DB041092DE04109240
:10282000DF041092E0041092E10488EF93E00E942C
:10283000760A2091D2043091D3044091D40450916F
:10284000D50486017501E21AF30A040B150BE6168E
:10285000F7060807190708F414C1A092D204B09231
:10286000D304C092D404D092D504809100089091F2
:1028700001088757974709F0A8958091E6048830AA
:10288000A0F08091C9039091CA03A091CB03B091AD
:10289000CC03FCE1B695A79597958795FA95D1F766
:1028A0000097A105B10509F08BC18091E6048F5F07
:1028B0008093E604E090D604F090D7040091D80409
:1028C0001091D904E114F1040105110511F188EF0B
:1028D00093E00E94760AAE18BF08C00AD10A6A15B2
:1028E0007B058C059D0588F48091C90384FD04C097
:1028F00080ED97E00E942D091092D6041092D70423
:102900001092D8041092D90404C080E090E00E9494
:102910002D0990910A05907C90930A05009152052B
:10292000109151050117B1F180915305823091F555
:10293000905890930A0588EF93E00E946C0A8930C2
:1029400010F048E002C0482F415030E013C03F5F14
:10295000A32FB0E0812F90E0FC01E85DFA4F2081C9
:10296000FD01E65FFA4F2083A85BBA4F2C930196D6
:10297000182F1F71341710F4101749F710935105D1
:10298000832F895C90910A05892B80930A053093E7
:1029900048051AC0209153052430D1F49091480580
:1029A000E9E4F5E0ABE0B5E0292F30E02E0F3F1F62
:1029B00002C081918D93E217F307D9F7995C80915A
:1029C0000A05982B90930A0583E08093530537C03E
:1029D0008091CD04823029F4916090930A055F9A2A
:1029E0000FC090930A055F98222319F481E0809329
:1029F000530580915305833019F484E08093530587
:102A0000F8940DEC13E07E010894E11CF11CF80130
:102A100081918F010E94E312F701819391937F01CD
:102A2000F3E00D3D1F0799F7809120048770BE01E8
:102A30006F5F7F4F4BE055E00E94FD0A7894469A05
:102A40008091CC040E944C0C88EF93E00E946C0AA9
:102A5000682F8AE095E00E940D11E091CC04EF5FB1
:102A6000E093CC04E83131F0F0E0E850FC4F87858A
:102A7000882339F41092CC0404C05F9A89E08093D3
:102A8000E60480912004887171F18091C203823044
:102A900051F58091E2049091E304880F991F90937F
:102AA000E3048093E20483E08093C2030E94000E5B
:102AB0000E94962A6093DE047093DF048093E00402
:102AC0009093E104611571058105910561F481E040
:102AD00090E0A0E0B0E08093DE049093DF04A09348
:102AE000E004B093E1048091200484FF1EC0809133
:102AF000E2049091E3048E7F0E94BF0B182F809117
:102B0000DA046091E4040E94FB0E082F8091DB043C
:102B1000612F0E94FB0E282F8091DC046091DD0460
:102B2000402F0091C3030E948C1246988091CD04DF
:102B30008130D1F0813020F0823009F047C034C0BC
:102B400082E10E94E12B892B09F040C081E0809353
:102B5000CD040E94882A6093CE047093CF048093A2
:102B6000D0049093D10432C082E10E94E12B892BE2
:102B700021F50E94882A2091CE043091CF04409103
:102B8000D0045091D104621B730B840B950B695ECA
:102B9000734080409040D0F082E08093CD0480ED7F
:102BA00097E00E942D0912C082E10E94E12B892B3F
:102BB00069F080E090E00E942D091092CD0406C0DB
:102BC0008091E604883009F059CF57CFA096EAE00B
:102BD0000C944A36219A229A23988BE060E00E9456
:102BE000362B8CE061E00E94362B089588E08093BC
:102BF000C1008AE061E00E94362B8AE060E00E941A
:102C0000AE2B0895ACE1B0E0E8E0F6E10C942E368E
:102C10000E94962A7B018C0181E00E94210D84E7AD
:102C2000A82E6E010894C11CD11CB3E0BB2EA98252
:102C3000C60161E00E944911B092C2030E94000ED9
:102C40006AEF70E080E090E00E94BC2A8091C203AD
:102C5000833009F07DC087E196E00E94122C892B19
:102C600009F076C00E94962A6E197F09800B910B9D
:102C70006058734C894C914008F06AC0D8CF8FE7F8
:102C80000E94170C0E942B0C843509F05CC08983CC
:102C90000E942B0C182F00E01093B4040093B3048F
:102CA0000E942B0C080F111D1093B4040093B30461
:102CB0000E942B0C8093B2040E942B0C8093B104D1
:102CC000813108F040C0FF2407C00E942B0C0F5632
:102CD0001B4FF8018083F3940F2D10E08091B10415
:102CE00090E0880F991F0817190778F380E7898308
:102CF000CE01019661E00E94491183E08093C203F6
:102D00000E94000E62E370E080E090E00E94BC2A26
:102D10008091C2038330A9F08FE70E94170C0E94B4
:102D20002B0C803581F489830DED13E00E942B0C70
:102D3000F80181938F01F3E0083F1F07B9F781E0A5
:102D400003C082E001C083E06C96EAE00C944A364E
:102D50008091C203833009F092CFF3CF83E00E94C9
:102D60003B0C8093210484E00E943B0C809322045E
:102D700087E061E00E94410C6AE070E080E090E052
:102D80000E94BC2A0E94000E000008950F931F931A
:102D9000082F17C05F9A64E670E080E090E00E9420
:102DA000BC2A5F9864E670E080E090E00E94BC2A54
:102DB0001F5F101778F36CE271E080E090E00E94F2
:102DC000BC2A10E0F6CF482F392F25E00DC0F99925
:102DD000FECF1FBA842F932F92BD81BD60BD0FB669
:102DE000F894FA9AF99A0FBE215059F0F999FECF4A
:102DF000842F932F92BD81BDF89A80B5681739F75B
:102E0000089582E00E94C6160895A0E0B0E0EBE0CD
:102E1000F7E10C942736482E562EEE24FF24882402
:102E20009924C0E0D0E0CC24DD2476E4372E04C021
:102E300055245394CC24DD24442069F48091C303A9
:102E4000839DE001112464ECE62E63E0F62E59E147
:102E5000852E912C1DC021E0421671F48091C30390
:102E6000839DE00111246B9648EFE42E43E0F42E9D
:102E700039E2832E912C0CC032E0431649F423EC46
:102E8000E22E23E0F22E91E0892E912CC8E1D1E0D0
:102E90003E016C0C7D1C10925C0510925B05E301F9
:102EA0001BC0552059F4F999FECFD2BDC1BDF89A87
:102EB00080B5F701E00FF11F808307C0F701E00F35
:102EC000F11FCE0160810E94E3160E0D1F1DF80157
:102ED00080810E94B10921969E012619022F10E0DF
:102EE00008151905F0F2CE015520D9F4F999FECF55
:102EF000D2BDC1BDF89A20B5F999FECF2196D2BDB9
:102F0000C1BD2197F89A80B590E0B22EAA248A29F3
:102F10009B2920915B0530915C052817390759F4EE
:102F200087CF219660915C050E94E316CE016091E7
:102F30005B050E94E31680E291E0C80ED91E91EE77
:102F4000C91692E0D90608F477CF852DCDB7DEB744
:102F5000E1E10C94433680E061E00E94051781E0D6
:102F600061E00E940517089580E060E00E94051767
:102F7000882331F081E060E00E940517882331F456
:102F80000E94130A0E94CE090E94AB17089582E0A6
:102F900061E00E940517089582E060E00E94051735
:102FA0008091C303843020F01092C3030E94C7179E
:102FB00008951F93182F0E94CC178091C303811787
:102FC00031F0143020F41093C3030E94C7171F91EF
:102FD00008951F93182F0E94962A6093C704709338
:102FE000C8048093C9049093CA041093B5041123B4
:102FF00029F440E855E260E070E004C040E051EEA2
:1030000060E070E08DEA96E00E94BB2F1F9108956A
:1030100087E196E0609128040E94732C08951F9325
:10302000182F87E196E0612F0E94732C809128046D
:103030008127809328041F9108951F93192F0E94C0
:103040000F18812F0E940F181F910895DF92EF92A1
:10305000FF920F931F93D82E7B011092280407E153
:1030600016E0C80165EB0E94732CC80162E60E945D
:10307000732C8D2D0E940F18C7010E941D181F91DF
:103080000F91FF90EF90DF90089510928F0485E6E6
:10309000EAE2F4E0DF011D928A95E9F708951F93B3
:1030A000182F8F3711F08830E1F5E0918F04EE236F
:1030B00009F455C0E150E0938F04F0E0E65DFB4F6A
:1030C000108287E196E06DE00E94732C10E00AC048
:1030D000E12FF0E0E65DFB4F87E196E060810E9422
:1030E000732C1F5F80918F04181790F387E196E08F
:1030F00060E20E94732C87E196E06DE00E94732CE1
:1031000010E00AC0E12FF0E0E65DFB4F87E196E0BA
:1031100060810E94732C1F5F80918F04181790F3B9
:103120001CC08B3119F40E9445181FC08D30E9F086
:103130008A30D9F080918F04843688F487E196E054
:10314000612F0E94732C80918F04E82FF0E0E65DE0
:10315000FB4F10838F5F80938F0480E007C087E16F
:1031600096E067E00E94692DF8CF81E01F910895F5
:103170001F93CF93DF93C7E0D4E010E03BC087E11B
:1031800096E062E271E00E94FA2E87E196E0612FFC
:103190004AE050E00E94772E87E196E06FE271E00E
:1031A0000E94FA2E699170E080E090E02091060480
:1031B00030E040E050E00E94B73520E137E240E0E7
:1031C00050E00E94B735DC01CB014091FD035091E6
:1031D000FE036091FF0370910004480F591F6A1F9E
:1031E0007B1F87E196E02AE030E00E943E2E1F5FC1
:1031F000183119F08881882311F6DF91CF911F9142
:103200000895EF92FF920F931F93882339F487E17B
:1032100096E061ED7AE00E94872D3BC090E00E942D
:10322000330A24E630E040E050E00E94E935122FF6
:10323000032FF42EE52E622F732F842F952F2AE073
:1032400030E040E050E00E94E93587E196E0BA01C5
:10325000A9012AE030E00E942F2E87E196E06EE27D
:103260000E94692D612F702F8F2D9E2D2AE030E056
:1032700040E050E00E94E935AB01BC0187E196E0F7
:103280002AE030E00E942F2E87E196E063E70E945B
:103290009B2D1F910F91FF90EF900895FF920F9338
:1032A0001F93CF93DF9387E196E067EC7AE00E946B
:1032B000482D8091DD03813041F487E196E06EEA8C
:1032C0007AE00E94872DFF246DC0823029F487E1C7
:1032D00096E067E97AE0F5CF843029F487E196E05B
:1032E00063E87AE0EECF853071F787E196E068E732
:1032F0007AE0E7CFCF2DD0E0C930D1051CF06F2D9B
:10330000685C02C06F2D6F5C87E196E00E94692DBA
:1033100087E196E060E77AE00E94482DBE016F5F8A
:103320007F4F87E196E04AE050E00E94D32E87E18C
:1033300096E065E67AE00E94482D8E0103521C4F0C
:10334000D8011196EC91E032F8F487E196E068E557
:103350007AE00E94482DF8018181803130F087E1C8
:1033600096E063E371E00E94FA2EC352DC4F69815C
:1033700070E06F7070706F5F7F4F87E196E04AE09A
:1033800050E00E94E62E0DC0F0E0EF70F070EE0FFE
:10339000FF1FEE5AFC4F6081718187E196E00E9429
:1033A000FD2EF3948091B204F81608F4A3CF87E1C0
:1033B00096E06DE37AE00E94482D8091F5030E942B
:1033C000011987E196E062E27AE00E94482D80913F
:1033D000F6030E94011987E196E067E07AE00E9417
:1033E000482D8091F7030E94011987E196E06CEE69
:1033F00079E00E94482D4091ED035091EE036091D9
:10340000EF037091F003411551056105710539F124
:1034100087E196E02AE030E00E943E2E87E196E0C8
:1034200069EB79E00E94482D8091F1030E94660AC1
:10343000AB01BC0187E196E02AE030E00E943E2E1D
:1034400087E196E065E979E00E94482D87E196E002
:103450006091F2034AE050E00E94892E06C087E1A5
:1034600096E06CE879E00E94872D87E196E06FE6B0
:1034700079E00E94482D6091F3037091F40387E195
:1034800096E04AE050E00E94632E87E196E062E514
:1034900079E00E94482D6091EC03603150F470E0B7
:1034A0006F5F7F4F87E196E04AE050E00E94E62E92
:1034B00006C087E196E069E479E00E94872D87E104
:1034C00096E06CE279E00E94482D8091EB0380FD4C
:1034D00003C065E371E002C069E371E087E196E053
:1034E0000E94FD2E87E196E06FE079E00E94482D72
:1034F0008091EB0382700E94050F87E196E060EFF8
:1035000078E00E94482D8091EB0384700E94050FA3
:1035100087E196E061ED78E00E94482D8091EB0311
:1035200088700E94050FCDB7DEB7E5E00C944F36EA
:103530001F93CF93DF9387E196E06BE17CE00E94DD
:10354000482D4091FD035091FE036091FF0370915F
:10355000000487E196E02AE030E00E943E2E87E1F9
:1035600096E065E07CE00E94482D40910104509176
:103570000204609103047091040487E196E020E165
:1035800030E00E943E2E87E196E06FEE7BE00E94E5
:10359000482D87E196E0609105044AE050E00E94E2
:1035A000892E87E196E069ED7BE00E94482D87E156
:1035B00096E0609106044AE050E00E94892E87E17F
:1035C00096E063EC7BE00E94482DC7E0D4E010E079
:1035D00012C0112331F087E196E06DE371E00E94A3
:1035E000FA2E87E196E069914AE050E00E94772E3A
:1035F0001F5F183119F08881882359F787E196E019
:103600000E94712D87E196E06DEA7BE00E94482DD3
:1036100087E196E060911F044AE050E00E94892E05
:1036200087E196E068E97BE00E94482DE091200464
:10363000F0E0E770F070EE0FFF1FEE58FC4F608176
:10364000718187E196E00E94FD2E87E196E063E8B4
:103650007BE00E94482D8091200490E0887190705A
:103660008830910589F0893091051CF4892B39F057
:103670001BC08031910569F04897B1F40FC087E114
:1036800096E06AE77BE00EC087E196E06EE67BE0BD
:1036900009C087E196E068E67BE004C087E196E038
:1036A0006EE57BE00E94872D87E196E06AE47BE08F
:1036B0000E94482D4091F9035091FA036091FB0359
:1036C0007091FC0387E196E02AE030E00E943E2EF4
:1036D00087E196E061E37BE00E94482D8091C90379
:1036E00080710E94050F87E196E068E17BE00E940F
:1036F000482D8091C90380740E94050F87E196E0F0
:103700006FEF7AE00E94482D8091C90380720E9479
:10371000050F87E196E062EE7AE00E94482D88EF7F
:1037200093E00E94760AAB01BC0187E196E02AE0B3
:1037300030E00E942F2E87E196E06DED7AE00E9446
:10374000482D88EF93E00E94760A9B01AC0160E46B
:1037500072E48FE090E00E94E93587E196E0BA01DB
:10376000A9012AE030E00E942F2E87E196E06AED61
:103770007AE00E94872DDF91CF911F910895EF92FB
:10378000FF920F931F938C0197E1E92E96E0F92E9B
:10379000C701612F70E04AE050E00E94522EC7013D
:1037A0006EE20E94692D84E0169507958A95E1F7EF
:1037B0000F701070C701B8014AE050E00E94522E0D
:1037C0001F910F91FF90EF9008950F931F93CF9348
:1037D000DF93209129042F3FA9F587E196E061E569
:1037E00076E00E94482D80E793E00E94BF1B87E1AE
:1037F00096E060E376E00E94482D8091B3049091BA
:10380000B4040E94BF1B87E196E06DEF75E00E9453
:10381000872D87E196E06AED75E00E94872D87E1AC
:1038200096E062EC75E00E94872D87E196E06DE9F5
:1038300075E00E94872D87E196E00E94712D0E941D
:103840004E1969C012160CF066C0332727FD30955B
:103850008091B20490E0821793070CF45CC087E17A
:1038600096E068E875E00E94482D6091290477276A
:1038700067FD709587E196E04AE050E00E94E62EF1
:1038800087E196E06DE575E00E94482D08E210E0C2
:103890003AC0C12FD0E0CC0FDD1FCF56DB4F2881BF
:1038A00030E080912904992787FD9095019728178A
:1038B000390741F587E196E06FE371E00E94FA2E47
:1038C00087E196E0602F4AE050E00E94772E87E182
:1038D00096E063E471E00E94FA2EE981F0E0EF7077
:1038E000F070EE0FFF1FEE5AFC4F6081718187E18F
:1038F00096E00E94FA2E87E196E067E471E00E946C
:10390000FA2E0F5F1F5F8091B104181710F287E144
:1039100096E00E94712DDF91CF911F910F91089534
:10392000ACE1B0E0E6E9FCE10C943036282F809160
:1039300029048F3F09F042C1822F90E0FC013A97A1
:10394000EF36F10508F033C1EA5AFF4F0C945D36AB
:1039500087E196E069E471E0AEC087E196E069E452
:1039600071E00E94FD2E1CC187E196E065E571E0E3
:103970000E94FD2E85E78983DE011296EDEDF3E0CE
:103980008BE101900D928150E1F7CE0101966CE13F
:103990000E9449110E94000E83E08093C20368ECEC
:1039A00070E080E090E00E94BC2A8091C2038430E5
:1039B00009F0FDC08FE70E94170C0E942B0C898331
:1039C000853509F0F4C087E196E06FE375E00E9469
:1039D000872D87E196E061E275E00E94872D87E1FF
:1039E00096E063E075E0ACC087E196E06DE671E0DB
:1039F0000E94FD2E89E68983CE01019661E00E9436
:103A000049110E94000E83E08093C20368EC70E0CD
:103A100080E090E00E94BC2A8091C203843009F0CB
:103A2000C6C08FE70E94170C0E942B0C89838E0161
:103A30000E5F1F4FFDE1EF2EF12CEC0EFD1E0E94DC
:103A40002B0CD8018D938D01AE15BF05C1F7ADEDDF
:103A5000B3E0FE0132968BE101900D928150E1F7C7
:103A60008981893409F0A3C087E196E065EE74E0AE
:103A70000E94872D87E196E067EC74E00E94872D15
:103A800087E196E069EA74E05BC087E196E067E869
:103A900071E00E94FD2E8EEF8093290488C0205291
:103AA0002750922F90538091B204891738F487E100
:103AB00096E066E971E00E94FD2E79C0909329049A
:103AC0006FC084E18093290487E196E062E774E0A7
:103AD00037C085E18093290487E196E06BE374E0C9
:103AE0002FC086E18093290487E196E064E074E0CA
:103AF00027C087E18093290487E196E06AEB73E0B1
:103B00001FC088E18093290487E196E069EA73E0A9
:103B100017C089E18093290487E196E065E973E0A5
:103B20000FC08AE18093290487E196E060E873E0A2
:103B300007C08BE18093290487E196E068E573E094
:103B40000E94872D34C087E196E06EE373E00E9407
:103B5000872D8091EB0391E01DC087E196E068E23C
:103B600073E00E94872D8091EB0392E013C087E100
:103B700096E063E173E00E94872D8091EB0394E06F
:103B800009C087E196E068EF72E00E94872D80917E
:103B9000EB0398E089278093EB038FEF8093290450
:103BA0000E94E51B04C087E196E00E94392C87E162
:103BB00096E00E94122C892BB1F763C1822F0E94DC
:103BC0004F18882309F45DC180918F04882321F464
:103BD0008FEF809329044DC18AE294E060E070E0A9
:103BE00040E050E00E94C3079B01AC0160912904B2
:103BF000862F992787FD9095A92FB92FFC01319722
:103C0000EB31F10508F025C1EB53FF4F0C945D3605
:103C1000E62FFF27E7FDF0958091B20490E08E1724
:103C20009F070CF416C1DA01C9010197A109B10976
:103C30008097A105B10540F0FF2410E008E26F0174
:103C40000894C108D10826C0E352FC4F822F81504E
:103C50008083E7C0612F70E0660F771F6F567B4F40
:103C6000FB01808190E08C159D0599F4802F90E0F8
:103C7000A0E0B0E082179307A407B50749F4F60166
:103C8000E352FC4FDB0111968C918183FF24F39466
:103C90000F5F1F5F8091B1041817E0F2C0C02F3F83
:103CA00031054105510511F008F0D3C02093F5030B
:103CB000B8C02F3F31054105510511F008F0C9C0CA
:103CC0002093F603AEC02F3F31054105510511F099
:103CD00008F0BFC02093F703A4C080912A0480623B
:103CE000803719F58BE294E060E070E040E050E04E
:103CF0000E94C3079B01AC01DC01CB010197A10924
:103D0000B1090897A105B10508F0B6C0CA01B9010B
:103D100024ED30E340E050E00E94B7359B01AC0158
:103D20002A5E3C4A4A46554E24C0863611F58BE23F
:103D300094E060E070E040E050E00E94C3079B0127
:103D4000AC01DC01CB010197A109B1090797A105DD
:103D5000B10508F091C0CA01B90128EA31E640E096
:103D600050E00E94B7359B01AC01245E3C434E46B7
:103D7000544E211531054105510561F0DA01C901A3
:103D8000805C9D49A845B54381509A45A246B24002
:103D900008F05FC02093ED033093EE034093EF03F0
:103DA0005093F0033EC02F3F31054105510511F0FE
:103DB00008F04FC02093F10334C0DA01C901019724
:103DC000A109B1098F3F9105A105B10508F041C0D6
:103DD0002093F20326C0DA01C901845C9940A04017
:103DE000B0408D549D41A040B04038F43093F4036E
:103DF0002093F303FF24F39401C0FF242115310520
:103E00004105510511F48FEF07C0213131054105FE
:103E1000510528F4822F81508093EC0302C0FF20CB
:103E2000C1F0809190048823D1F480910104909195
:103E30000204A0910304B09104040196A11DB11DD8
:103E40008093010490930204A0930304B0930404AC
:103E500006C087E196E068EA71E00E94FD2E0E94AC
:103E600045188FEF8093290487E196E06AE00E946D
:103E70009B2D0E94E51B05C021E030E040E050E0B2
:103E80007DCF6C96E8E00C944C3687E196E06CEAC6
:103E900072E00E94872D87E196E064E972E00E945B
:103EA000872D87E196E00E94122C892B31F087E163
:103EB00096E00E94392C0E94901C0E9402168230CB
:103EC00019F0833069F405C087E196E066E772E097
:103ED00004C087E196E06FE572E00E94872D0895A7
:103EE0008FEF80932904109290040E94E51B0CC070
:103EF00087E196E00E94122C892B31F087E196E051
:103F00000E94392C0E94901C809129048E3F81F7D9
:103F1000089580912904992787FD9095A92FB92F9D
:103F2000FC013196EB30F10508F074C0E052FF4F10
:103F30000C945D3687E196E064EC78E00E94872D72
:103F400080E793E00E94BF1B87E196E06CEA78E08F
:103F50000E94872D87E196E067E878E00E94872D30
:103F600087E196E06DE578E00E94872D87E196E095
:103F70006CE378E00E94872D87E196E06FE078E0BF
:103F80000E94872D87E196E069EE77E00E94872DF9
:103F900087E196E065EC77E00E94872D87E196E067
:103FA0006EE977E00E94872D87E196E00E94712DEF
:103FB0000E94981A2FC087E196E061E877E028C058
:103FC00087E196E06CE577E023C087E196E067E45F
:103FD00077E01EC087E196E068E277E019C087E1EC
:103FE00096E064EE76E014C087E196E06FEC76E050
:103FF0000FC087E196E06AEB76E00E94872D87E1AB
:1040000096E064E776E004C087E196E06EE576E04E
:104010000E94872D6AE070E080E090E00E94BC2A58
:1040200004C087E196E00E94392C87E196E00E9467
:10403000122C892BB1F70895A2E2B0E0E2E2F0E29F
:104040000C9426368E010F5F1F4F80E1D8011D9220
:104050008A95E9F787E196E066EC71E00E94FD2E13
:104060000E94AE1620EC3DE948E555E32F8F38A3BA
:1040700049A35AA380EC97EFAAEBB7E38B8F9C8FF1
:10408000AD8FBE8F24EF31E040E050E02F8B388FB2
:10409000498F5A8F90E5C92E93ECD92EE12CF12C43
:1040A00080EC482E8DE9582E88E5682E85E3782E21
:1040B00088249924540133241E8A1D8A198A1A8A55
:1040C0001B8A1C8AFFC087E196E00E94392C843449
:1040D000B9F0853430F48332B9F18C3209F0CCC0B8
:1040E00044C0833509F0C8C02F8D38A149A15AA119
:1040F000C901DA012C013D01882499245401E2C050
:1041000087E196E064E40E94692D87E196E040EC47
:104110005DE968E575E32AE030E00E949D2E87E1C5
:1041200096E06CE20E94692D87E196E040EC57EF43
:104130006AEB77E32AE030E00E949D2E87E196E06B
:104140006CE20E949B2DBEC019821A821B821C82C7
:104150001D821E821F82188619861A861B861C865F
:104160001D861E861F86188A3AC0339434E03316A3
:1041700009F0A8C069817A818B819C8128EE33E0A7
:1041800040E050E00E94B7356F8F78A389A39AA3CF
:104190006D817E818F8198850E94B7356B8F7C8F72
:1041A0008D8F9E8F89859A85AB85BC858F8B988FE7
:1041B000A98FBA8F6D857E858F8598890E94B735C6
:1041C0006B017C0190E2C9169EE4D90690E0E906F5
:1041D00090E0F90630F48CE162E30E94410C332454
:1041E00071C0A0E3CA16A5E7DA06A0E0EA06A0E0DF
:1041F000FA0618F48CE162E2F0CFB0E4CB16BCE929
:10420000DB06B0E0EB06B0E0FB0618F48CE166E2FA
:10421000E4CFE0E5CE16E3ECDE06E0E0EE06E0E01B
:10422000FE0618F48CE162E1D8CFF0E6CF16FAEE84
:10423000DF06F0E0EF06F0E0FF0618F48CE165E140
:10424000CCCF20E7C21621E1D20621E0E20620E031
:10425000F20618F48CE161E0C0CF30EAC31636E80C
:10426000D30631E0E30630E0F30618F48CE163E0B6
:10427000B4CF8CE165E0B1CFB0ED2B2E280E49E034
:10428000421500F1032D10E0000F111F000F111F48
:1042900081E090E08C0F9D1F080F191FD8016D91D0
:1042A0007D918D919C912AE030E040E050E00E94A9
:1042B000B735620D711D811D911DF80160837183F9
:1042C0008283938387E196E00E94122C892B09F068
:1042D000FACE81149104A104B10489F4C301B2019E
:1042E0000E94B70C61E070E080E090E00E94BC2A80
:1042F000FFEFFE8B1D8A198A1A8A1B8A1C8A2F8956
:10430000388D498D5A8D82169306A406B506E0F4C1
:104310000E94620C29893A894B895C89280F311DDA
:10432000411D511D298B3A8B4B8B5C8B3D89381776
:1043300008F48D8B4E89841708F48E8B0894811CA9
:10434000911CA11CB11C56C0C301B20128EE33E080
:1043500040E050E00E94E93587E196E0BA01A9010A
:104360002AE030E00E942F2E87E196E06CE20E9466
:10437000692D87E196E06D894AE050E00E94772E32
:1043800087E196E06CE20E94692D69897A898B89C0
:104390009C89A50194010E94E93587E196E0BA0164
:1043A000A9012AE030E00E942F2E87E196E06CE21E
:1043B0000E94692D87E196E06E894AE050E00E94F4
:1043C000772E87E196E06CE20E949B2D4C0C5D1CE1
:1043D0006E1C7F1C8B8D9C8DAD8DBE8D84159505BF
:1043E000A605B70520F44F8C58A069A07AA08824B0
:1043F000992454012F8D38A149A15AA1285E334038
:104400004040504009F05ECFA296E2E10C94423663
:10441000AAE5B0E0EEE0F2E20C9432368B017A01CC
:104420008B3009F426C18C3040F5853009F484C006
:10443000863080F4823009F459C0833020F4813012
:1044400009F052C242C0833009F461C0843009F0DF
:104450004BC265C0883009F49DC0893038F486307D
:1044600009F486C0873009F03FC28CC0893009F456
:1044700099C08A3009F038C2C9C0893609F484C1AC
:104480008A3680F4863609F42FC1873620F48536C3
:1044900009F02AC210C1873609F43FC1883609F0F5
:1044A00023C243C18C3609F4C6C18D3638F48A362E
:1044B00009F475C18B3609F017C2B1C18D3609F404
:1044C000EEC1873C09F010C202C281E069E270E0EF
:1044D0000E94261808EF13E0F80181918F010E94D5
:1044E0000F18F4E001321F07B9F706C282E06BE152
:1044F00070E00E9426180DED13E0F80181918F0104
:104500000E940F18F3E0083F1F07B9F7F5C183E0D9
:1045100061E070E00E9426180E940216EBC184E060
:1045200061E070E00E94261881E00E940F180E944E
:1045300008180E941C20E2C16091B10470E0660F6F
:10454000771F85E00E94261800E010E008C0F801FF
:10455000EF56FB4F80810E940F180F5F1F4F809115
:10456000B10490E0880F991F0817190780F3C4C1A0
:1045700086E062E070E00E94261880E793E00E94E7
:104580001D18BAC187E061E070E00E942618809192
:10459000B204B0C188E061E070E00E94261880910A
:1045A000C303A8C186E68983CE01019661E00E941B
:1045B00049110E94000E83E08093C20368EC70E012
:1045C00080E090E00E94BC2A8091C2038430E1F434
:1045D0008FE70E94170C0E942B0C8983863471F49C
:1045E00089E060E270E00E94261810E00E942B0C27
:1045F0000E940F181F5F1032C9F77EC189E061E089
:1046000070E00E942618C9C089E06FC18AE069E1A4
:1046100070E00E94261882E08093C4038091C9054F
:10462000882351F08091C9039091CA03A091CB03D4
:10463000B091CC03806809C08091C9039091CA03EE
:10464000A091CB03B091CC038F778093C903909353
:10465000CA03A093CB03B093CC0304EC13E0F8019E
:1046600081918F010E940F18F3E00D3D1F07B9F7EC
:1046700043C18BE061E270E00E9426188091E6045D
:104680008F3F39F08091E6048F5F8093E60481507C
:1046900002C08091E6040E940F1810E0F894812F68
:1046A0000E94E3120E949A0B0E941D1878941F5FCB
:1046B0001031A1F721C185E661E070E00E94261863
:1046C0000932110509F015C120E030E0F901E85088
:1046D000FC4FD701A20FB31F8C9180832F5F3F4FF8
:1046E0002932310599F759C086E661E070E00E94F1
:1046F00026180B31110509F0FCC020E030E0F9016B
:10470000E352FC4FD701A20FB31F8C9180832F5F20
:104710003F4F2B31310599F740C087E661E070E0EB
:104720000E9426180E94AB1738C088E661E070E04E
:104730000E94261885E78A83DE011396EDEDF3E0EB
:104740008BE101900D928150E1F7CE0102966CE170
:104750000E9449110E94000E83E08093C20360E230
:1047600073E080E090E00E94BC2A8091C203843014
:1047700009F0BFC08FE70E94170C0E942B0C8A83A0
:10478000853509F0B6C009C089E661E070E00E9495
:1047900026180E94CE090E94130A81E0ABC08AE667
:1047A00061E070E00E94261889E68E8FCE014E9659
:1047B00061E00E9449110E94000E83E08093C203D1
:1047C00060E273E080E090E00E94BC2A8091C20326
:1047D000843009F08EC08FE70E94170C0E942B0CCA
:1047E0008E8F8E01015E1F4F2AE3E22EF12CEC0E1C
:1047F000FD1E0E942B0CF80181938F01EE15FF0521
:10480000C1F7ADEDB3E0FE017F968BE101900D9213
:104810008150E1F78E8D893409F06BC0BECF8BE6F5
:1048200061E070E00E942618F70180810E94D9178C
:104830000E94B417B2CF8CE661E070E00E942618A7
:104840000032110571F487E68AAFDE01DB96F701CD
:1048500080E201900D928150E1F7CE01CA9661E2AB
:1048600005C087E48AAFCE01CA9661E00E94491173
:104870000E94000E83E08093C2036CE474E080E049
:1048800090E00E94BC2A8091C203843091F58FE7AA
:104890000E94170C0E942B0C873459F57ECF8DE6B1
:1048A00061E070E00E9426180931110511F520E041
:1048B00030E0F901EC53FC4FD701A20FB31F8C91EC
:1048C00080832F5F3F4F2931310599F766CF87EC01
:1048D00061E070E00E94261881E00E940F180E949B
:1048E0000818109227040AC08AEC61E070E00E9468
:1048F000261880E00E940F180E940818C65ADF4F41
:10490000E6E00C944E36A0E0B0E0E9E8F4E20C9466
:104910002E36A4E0AA2EF6E0BF2EE5E0CE2E0DE561
:1049200015E074E6D72E62E0E62E53E0F52EA1C026
:1049300087E196E00E94392C982F8093C8058091DA
:10494000C705833021F1843028F4813099F082301A
:10495000B8F409C0853009F448C0853020F18630AC
:1049600009F087C05FC0953B09F083C081E0809368
:10497000C7057FC0923609F07AC0E092C70579C0BA
:104980009093C6059093C505F092C70572C09093A9
:10499000C3051092C4058091C50589278093C5057C
:1049A000A092C70566C0D92FC0E02091C305309101
:1049B000C4052C2B3D2B3093C4052093C305809157
:1049C000C50589278093C505C092C70525363105E1
:1049D00008F44FC08CEC61E070E00E94261881E082
:1049E0000E940F180E94081842C02091C105309102
:1049F000C205F901E35AFA4F90838091C5058927D2
:104A00008093C5052F5F3F4F3093C2052093C105AA
:104A10008091C3059091C4052817390750F1B092D1
:104A2000C70527C08091C505891759F46091C10554
:104A30007091C2058091C6054DE555E00E9408229F
:104A40000DC08BEC62E070E00E9426188091C605D4
:104A50000E940F18809128040E940F18F8018D2DD4
:104A600011928A95E9F71092C2051092C105109231
:104A7000C70587E196E00E94122C892B09F058CFD8
:104A8000CDB7DEB7EAE00C944A3681E08093270484
:104A900008C087E196E00E94122C892B11F00E9439
:104AA0008324809127048823A1F70895A0E0B0E033
:104AB000ECE5F5E20C9431360E94962A61157105F9
:104AC00081059105C9F30E94BA0710920104109262
:104AD00002041092030410920404DD24E090010407
:104AE000F09002040091030410910404102F0F2D84
:104AF000FE2CEE240E94B5072FEF30E040E050E09E
:104B00000E940B36E60EF71E081F191FE0920104E3
:104B1000F09202040093030410930404D39444E03D
:104B2000D416E1F6C7E0D4E000E010E0B0E1EB2EEF
:104B3000B7E2FB2E4EC00F5F19F40E94CE094DC0A4
:104B40000E94B50722E330E040E050E00E940B36BF
:104B50006F5FE7E0F4E090E004C08191861759F3BD
:104B60009F5F9117D0F38091060490E08E9D900195
:104B70008F9D300D9E9D300D1124862F90E0AC014D
:104B8000249FC001259F900D349F900D1124AA27CA
:104B900097FDA095BA2F2091FD033091FE0340911F
:104BA000FF0350910004820F931FA41FB51F209193
:104BB000C5033091C6034091C7035091C80328171D
:104BC00039074A075B0708F4B6CF69931F5F1831AE
:104BD00021F08881882309F0AECFCDB7DEB7E7E0BA
:104BE0000C944D361F93109129041F3F09F0F1C01A
:104BF000893409F467C08A3428F5883309F479C008
:104C0000893368F4803309F486C0813308F06FC0BB
:104C10008B3109F44DC0813209F0D5C03DC08134DB
:104C200009F49AC0823438F4893309F472C08034AC
:104C300009F0C9C031C0823409F4A1C0863409F03A
:104C4000C2C052C0823609F49AC0833690F48835C7
:104C500079F1893538F4823509F43FC0833509F09C
:104C6000B2C01FC08A3509F4A9C0813609F0ABC0B3
:104C700073C0823791F1833730F48636A9F18936D3
:104C800009F0A1C01FC0883799F08A3709F496C08F
:104C9000833709F098C005C087E196E069E471E0C8
:104CA00019C00E94AB1787E196E063ED71E006C082
:104CB0000E94B41787E196E06DEE71E00E94FD2E30
:104CC0008EEF7FC00E94CE090E94130A87E196E012
:104CD0006CE072E00E94FD2E76C00E94562587E1AE
:104CE00096E065E272E0F6CF0E94B8186CC080537F
:104CF00068C087E196E06CE472E00E94872D909195
:104D00002004892F885F8871977E892B80932004E7
:104D100020C089E056C087E196E069E372E00E9416
:104D2000872D8091C9039091CA03A091CB03B091C4
:104D3000CC0320E130E040E050E082279327A42715
:104D4000B5278093C9039093CA03A093CB03B09374
:104D5000CC031093290437C087E196E063E272E048
:104D60000E94872D8091C9039091CA03A091CB0323
:104D7000B091CC0320E430E040E050E012C087E185
:104D800096E062E172E00E94872D8091C9039091C4
:104D9000CA03A091CB03B091CC0320E230E040E005
:104DA00050E082279327A427B5278093C9039093C7
:104DB000CA03A093CB03B093CC0302C00E94451F4B
:104DC0008FEF80932904809129048E3F09F4DDC080
:104DD000D4C00E944F18882309F4D7C080918F0453
:104DE000882321F48FEF80932904C7C08AE294E0DE
:104DF00060E070E040E050E00E94C3079B01AC011E
:104E000080912904992787FD9095A92FB92FFC013E
:104E10003197E930F10508F08CC0E551FF4F0C9453
:104E20005D36DA01C901815C9D49A845B5438F5FB4
:104E30009945A246B24008F07CC02093FD03309310
:104E4000FE034093FF03509300049AC02093010493
:104E500030930204409303045093040481E0809350
:104E600090048EC0283031054105510508F061C01D
:104E70002093050485C0DA01C9010197A109B10990
:104E80000A97A105B10508F054C02093060478C024
:104E90008AE294E06DE371E00E94DF0810E00EC04A
:104EA000183130F4E12FF0E0E850FC4F87871F5FA6
:104EB00080E090E06DE371E00E94DF08009759F018
:104EC0000E94C108009761F706C0E12FF0E0E850AA
:104ED000FC4F17861F5F1831C0F352C025303105D3
:104EE0004105510530F520931F044AC0DA01C9017C
:104EF0000197A109B1090697A105B105D0F48091E8
:104F00002004887F822B809320043AC0DA01C901F3
:104F10000197A109B1098050924CA140B04048F4DA
:104F20002093F9033093FA034093FB035093FC035F
:104F300027C087E196E068EA71E00E94FD2E13C069
:104F40008091010490910204A0910304B0910404A3
:104F50000196A11DB11D8093010490930204A093BA
:104F60000304B09304040E9445188FEF8093290432
:104F700087E196E06AE00E949B2D0E94891F05C090
:104F8000809190048823E1F2EECF1F9108958FEF76
:104F900080932904109290040E94891F0CC087E11D
:104FA00096E00E94122C892B31F087E196E00E9456
:104FB000392C0E94F225809129048E3F81F76AE006
:104FC00070E080E090E00E94BC2A04C087E196E097
:104FD0000E94392C87E196E00E94122C892BB1F7B0
:104FE0000895AAE2B0E0E7EFF7E20C942B360E94B6
:104FF000882A7B018C0181E00E94210D04C087E199
:1050000096E00E94392C87E196E00E94122C892BB1
:10501000B1F75F98DD24D39432E6732E22E0822E1E
:10502000912C8C0E9D1E5E010894A11CB11C93E076
:10503000C92E0E94882A20E030E06E197F09800B7B
:10504000910B693C71058105910510F021E030E07C
:105050008D2D90E028233923232B99F10E94882A53
:105060007B018C01469A80ED97E00E942D097982A0
:10507000D401E8EFF3E089E201900D928150E1F76D
:10508000C5016AE20E944911469880E090E00E94C2
:105090002D09C092C2030E94000E62E370E080E01E
:1050A00090E00E94BC2A8091C203843051F4C092E7
:1050B000C2038FE70E94170C0E942B0C823409F464
:1050C000DD2482E10E94E12B892B49F5DD24D39474
:1050D00026C05F9A469A87E196E00E94392C8D306F
:1050E000910569F08E3091051CF40A97B1F407C060
:1050F0008332910569F08234910579F40CC087E11F
:1051000096E064E072E00E94872D0E94C72705C0E8
:105110000E941C2002C00E9445255F98469887E1A6
:1051200096E00E94122C892B09F483CFD2CF8F9264
:105130009F92AF92BF92CF92DF92EF92FF920F9326
:105140001F9382E10E94E12B892B09F083C068EC58
:1051500070E080E090E00E94BC2A80E090E00E9435
:105160002D090E94882A5B016C0140ECE42E42E18B
:10517000F42E012D112DE60EF71E081F191F06C073
:1051800082E10E94E12B892B09F062C00E94882AEB
:105190006E157F058007910798F382E10E94E12B4D
:1051A000892B09F055C080ED97E00E942D090E94DF
:1051B000882A7B018C0188249924939488E496E2C0
:1051C000A0E0B0E0A80EB91ECA1EDB1E29C0AE14B6
:1051D000BF04C006D10638F480ED97E00E942D0987
:1051E000882483941DC00E94882A6E197F09800B31
:1051F000910B693C71058105910590F00E94882A08
:105200007B018C0180E0992009F481E0982E8823AD
:1052100019F480E090E002C080ED97E00E942D0933
:1052200082E10E94E12B892B91F280E090E00E94C4
:105230002D09882049F08091C3038F5F83700E94FD
:10524000D9170E94B41706C00E9456250E94AB17BA
:105250000E94F1271F910F91FF90EF90DF90CF9068
:10526000BF90AF909F908F900895EF92FF920F9311
:105270001F9380E00E948C090E94EA1586E061E09D
:105280000E94362B85E061E00E94362B82E160E0CF
:105290000E94362B84E060E00E94362B84E061E0BF
:1052A0000E94AE2B0E94F61587E196E060E070E068
:1052B0000E94112C0E94CC170E94B4170E94E00E8D
:1052C0008FEF8093E6040E94590978940E94882AFF
:1052D0007B018C018091E6048F3F09F0C7C00E94DA
:1052E000882A6E197F09800B910B605D77408040A2
:1052F000904008F0BBC0EECF87E196E00E94392CC9
:1053000087E196E00E94122C892BB1F787E196E0A5
:1053100062E472E00E94FA2E80E793E00E94BF1BD5
:1053200087E196E069E572E00E94FA2E87E196E057
:1053300066E070E04AE050E00E94E62E62E370E032
:1053400080E090E00E94BC2A87E196E00E94122C47
:1053500004970CF187E196E00E94392C8234910584
:10536000D1F487E196E00E94392C8E34910599F4AE
:1053700087E196E00E94392C8434910561F487E13D
:1053800096E00E94392C819731F480E090E00E94F1
:105390002D090E94F1274091F9035091FA03609181
:1053A000FB037091FC03DB01CA010197A109B1095C
:1053B0000497A105B10568F44093E704433029F050
:1053C00040E052EC61E070E004C040EA56E861E081
:1053D00070E08DEA96E00E94BB2F0E9497285F98AC
:1053E00080E090E00E942D090E94E00E80E00E9483
:1053F000210D8091CC040E944C0C0E94000E109252
:105400005105109252051092530510E015C062E349
:1054100070E080E090E00E94BC2A80ED97E00E945E
:105420002D0962E370E080E090E00E94BC2A80E0F9
:1054300090E00E942D091F5F8091C303811738F708
:105440008091200490E084FF09C020E08871907072
:10545000489709F421E0822F0E94E9178FE00E940B
:105460008C091F910F91FF90EF90089580ED97E0C8
:105470000E942D0982E161E00E94AE2B5F9A40CF2D
:105480001F920F920FB60F9211242F933F938F9379
:105490009F93AF93BF938091CE059091CF05A0913C
:1054A000D005B091D1053091D2050196A11DB11D55
:1054B000232F2D5F2D3720F02D570196A11DB11DF3
:1054C0002093D2058093CE059093CF05A093D0056D
:1054D000B093D1058091CA059091CB05A091CC05E0
:1054E000B091CD050196A11DB11D8093CA05909381
:1054F000CB05A093CC05B093CD05BF91AF919F9103
:105500008F913F912F910F900FBE0F901F90189584
:105510008FB7F8942091CE053091CF054091D005FA
:105520005091D1058FBFB901CA0108959FB7F89472
:105530002091CA053091CB054091CC055091CD0505
:1055400086B5A89B06C08F3F21F02F5F3F4F4F4F7E
:105550005F4F9FBF542F432F322F2227280F311D1B
:10556000411D511D82E0220F331F441F551F8A9594
:10557000D1F7B901CA010895EF92FF920F931F93DB
:10558000CF93DF937B018C010E94962AEB010EC022
:105590000E94962A6C1B7D0B685E7340C8F30894CA
:1055A000E108F10801091109C851DC4FE114F104C7
:1055B0000105110569F7CDB7DEB7E6E00C944E366C
:1055C000789484B5826084BD84B5816084BD85B5DE
:1055D000826085BD85B5816085BDEEE6F0E08081A5
:1055E00081608083E1E8F0E01082808182608083C6
:1055F000808181608083E0E8F0E080818160808349
:10560000E1E9F0E080818260808380818160808335
:10561000E0E9F0E0808181608083E1ECF0E080816E
:1056200084608083808182608083808181608083C8
:10563000E3ECF0E0808181608083E0ECF0E0808149
:1056400082608083E2ECF0E0808181608083EAE721
:10565000F0E08081846080838081826080838081AB
:10566000816080838081806880830895CF93DF93F9
:10567000482F50E0CA018758934FFC013491455A96
:10568000534FFA018491882369F190E0880F991FA4
:10569000FC01EF5CF34FA591B491FC01E15CF34F89
:1056A000C591D491662351F42FB7F8948C91932F20
:1056B000909589238C93888189230BC0623061F493
:1056C0002FB7F8948C91932F909589238C93888190
:1056D000832B88832FBF06C09FB7F8948C91832BB0
:1056E0008C939FBFDF91CF91089590E0FC0131979B
:1056F000EE30F10590F5EC50FF4F0C945D36809143
:1057000080008F7703C0809180008F7D8093800020
:10571000089584B58F7702C084B58F7D84BD0895C8
:10572000809190008F7707C0809190008F7D03C09B
:1057300080919000877F8093900008958091C000B1
:105740008F7703C08091C0008F7D8093C000089543
:105750008091C200877F8093C2000895FF920F93CB
:105760001F93F62E482F50E0CA018956934FFC0133
:105770002491CA018758934FFC011491455A534F05
:10578000FA0104910023C9F0222319F0822F0E940C
:10579000752BE02FF0E0EE0FFF1FE15CF34FA591BA
:1057A000B4919FB7F894FF2021F48C911095812338
:1057B00002C08C91812B8C939FBF1F910F91FF9002
:1057C00008950F931F93482F50E0CA018956934FB5
:1057D000FC012491CA018758934FFC010491455A5A
:1057E000534FFA011491112319F420E030E015C051
:1057F000222319F0822F0E94752B812F90E0880FB1
:10580000991F835B934FFC01A591B4918C9120E08B
:1058100030E0802311F021E030E0C9011F910F91A9
:10582000089508952091130630911406809115066D
:1058300090911606281B390B2F733070C9010895FB
:10584000209113063091140680911506909116064A
:105850002817390719F42FEF3FEF09C0E09115061B
:10586000F0911606ED52FA4F8081282F30E0C901E1
:105870000895209113063091140680911506909199
:1058800016062817390719F42FEF3FEF13C0E091E0
:105890001506F0911606ED52FA4F208180911506FB
:1058A0009091160601968F739070909316068093D0
:1058B000150630E0C901089510921A0610921906D3
:1058C00088EE93E0A0E0B0E080931B0690931C0666
:1058D000A0931D06B0931E0684E993E090931806EA
:1058E000809317060895A1E0B0E0E9E7FCE20C948C
:1058F00034368C01698380914F03882369F083E0FB
:10590000BE016F5F7F4F41E050E00E945032181699
:10591000190614F49C0107C081E090E0F80193831C
:10592000828320E030E0C9012196E4E00C945036F7
:1059300083E00E9427320895CF93DF9312C082E064
:105940000E9497312FEF8F3F9207C9F0E091130625
:10595000F0911406ED52FA4F8083D0931406C09351
:105960001306C0911306D09114062196CF73D07000
:105970008091150690911606C817D90701F7DF9197
:10598000CF910895FC0180818E5F808380E861EC77
:105990007CE042E450E00E94CE310895FC01818118
:1059A0009081913A59F4813209F04CC080E068E46A
:1059B00073E047E050E00E94CE3142C0913209F0DE
:1059C00041C0803239F488E493E067E070E00E94DF
:1059D000123236C0823209F035C0828180934F0383
:1059E0008091480390914903A0914A03B0914B03E1
:1059F000805B9440A040B04019F580914F0380FD3A
:105A000012C087E797E790930108809300082BE086
:105A100088E190E00FB6F894A895809360000FBEDF
:105A2000209360000DC088E10FB6F8948093600069
:105A3000109260000FBEA895109201081092000805
:105A400081E0089580E00895A0E0B0E0EAE2FDE2A0
:105A50000C9430367C016B018A01C0E0D0E00FC0AD
:105A6000D6016D916D01D701ED91FC910190F0810E
:105A7000E02DC7010995C80FD91F0150104001152D
:105A8000110571F7CE01CDB7DEB7E8E00C944C36C6
:105A9000EF92FF920F931F93CF93DF937C018B01C3
:105AA000C0E0D0E0F8010F5F1F4F6491662359F00A
:105AB000D701ED91FC910190F081E02DC70109958E
:105AC000C80FD91FEFCFCE01CDB7DEB7E6E00C94FB
:105AD0004E36DC01ED91FC910190F081E02D0995AD
:105AE0000895EF92FF920F931F938C016DE00E9437
:105AF000692D7C01C8016AE00E94692D9C012E0D70
:105B00003F1DC9011F910F91FF90EF900895EF92F3
:105B1000FF920F931F937C010E94482D8C01C701B7
:105B20000E94712D9C01200F311FC9011F910F91FF
:105B3000FF90EF900895EF92FF920F931F937C01D7
:105B40000E94692D8C01C7010E94712D9C01200FBC
:105B5000311FC9011F910F91FF90EF900895CF93CE
:105B6000DF93EC016115710519F420E030E00FC0FE
:105B7000DB010D900020E9F71197A61BB70BE88118
:105B8000F9810280F381E02DAD0109959C01C901E5
:105B9000DF91CF9108954F925F927F928F929F9263
:105BA000AF92BF92CF92DF92EF92FF920F931F932B
:105BB000DF93CF93CDB7DEB7A1970FB6F894DEBFD2
:105BC0000FBECDBF2C01742ECB01223008F42AE089
:105BD00019A231E2C32ED12CCC0EDD1E822E9924C7
:105BE000AA24BB24672D752FA50194010E94E935D5
:105BF00079018A01C801B701A50194010E94B73556
:105C0000472D461B0894C108D1084A3010F4405D66
:105C100001C0495CF6014083E114F104010511055E
:105C200021F07E2C5F2DC801DDCFC201B6010E949C
:105C3000AF2DA1960FB6F894DEBF0FBECDBFCF91AA
:105C4000DF911F910F91FF90EF90DF90CF90BF9069
:105C5000AF909F908F907F905F904F900895DC0160
:105C60002115310541F4ED91FC910190F081E02D79
:105C7000642F099508950E94CB2D0895EF92FF920D
:105C80000F931F937C010E942F2E8C01C7010E944D
:105C9000712D9C01200F311FC9011F910F91FF90A1
:105CA000EF900895EF92FF920F931F939A017B015B
:105CB00000E010E0B801A7010E942F2E1F910F9164
:105CC000FF90EF900895EF92FF920F931F937C0146
:105CD0000E94522E8C01C7010E94712D9C01200F41
:105CE000311FC9011F910F91FF90EF900895EF921E
:105CF000FF920F931F939A01E62EFF2400E010E01D
:105D0000B801A7010E942F2E1F910F91FF90EF90D5
:105D10000895EF92FF920F931F937C010E94772EBC
:105D20008C01C7010E94712D9C01200F311FC901F8
:105D30001F910F91FF90EF900895A0E0B0E0E3EA8B
:105D4000FEE20C943036EC016A017B01211531052D
:105D500041F4E881F9810190F081E02D642F0995EB
:105D60001BC02A303105B1F477FF13C06DE20E94E9
:105D7000692D8C0144275527BA014C195D096E091C
:105D80007F09CE012AE00E94CB2D9C01200F311FFC
:105D900004C02AE00E94CB2D9C01C901CDB7DEB71B
:105DA000E8E00C944C36EF92FF920F931F937B0127
:105DB0009A010027F7FC0095102FB801A7010E9457
:105DC0009D2E1F910F91FF90EF900895EF92FF92FB
:105DD0000F931F937C010E94D32E8C01C7010E9458
:105DE000712D9C01200F311FC9011F910F91FF9050
:105DF000EF9008950E94AF2D0895EF92FF920F93B8
:105E00001F937C010E94FA2E8C01C7010E94712D04
:105E10009C01200F311FC9011F910F91FF90EF903E
:105E2000089508951F920F920FB60F9211242F9389
:105E30003F934F938F939F93EF93FF938091C8006D
:105E400082FD1DC04091CE0020916506309166060E
:105E50002F5F3F4F2F7330708091670690916806D7
:105E60002817390771F0E0916506F0916606EB5D41
:105E7000F94F4083309366062093650602C08091F7
:105E8000CE00FF91EF919F918F914F913F912F9174
:105E90000F900FBE0F901F9018951F920F920FB684
:105EA0000F9211242F933F938F939F93EF93FF9320
:105EB0002091A9063091AA068091AB069091AC067C
:105EC0002817390731F48091C9008F7D8093C9006C
:105ED00014C0E091AB06F091AC06E759F94F208170
:105EE0008091AB069091AC0601968F739070909361
:105EF000AC068093AB062093CE00FF91EF919F916B
:105F00008F913F912F910F900FBE0F901F9018957A
:105F1000A0E0B0E0EEE8FFE20C942C36FC01138226
:105F2000128288EE93E0A0E0B0E084839583A6839C
:105F3000B78386EA93E09183808375876487578768
:105F40004687318B208B138B028BF58AE48AD78AA4
:105F5000C68AB18EA08E938E828E8F85848F88891B
:105F6000858F8989868F8A89878F8B8980A32096E0
:105F7000ECE00C944836AF92BF92DF92EF92FF9222
:105F80000F931F93CF93DF93EC017A018B01DD24F4
:105F9000403081EE580780E0680780E0780711F014
:105FA000DD24D39491E0A92EB12CEC89FD89DD206C
:105FB00069F0C50108A002C0880F991F0A94E2F792
:105FC000808360E079E08DE390E005C0108260E8B6
:105FD00074E88EE190E0A80197010E94E935215014
:105FE000304040405040569547953795279580E181
:105FF0002030380720F0DD2011F0DD24D6CFE889ED
:10600000F9893083EA89FB89208319A2EE89FF8907
:10601000408121E030E0C9010C8C02C0880F991F3B
:106020000A94E2F7482B4083EE89FF894081C90139
:106030000D8C02C0880F991F0A94E2F7482B408309
:10604000EE89FF894081C9010E8C02C0880F991F1B
:106050000A94E2F7482B4083EE89FF8980810F8CF8
:1060600002C0220F331F0A94E2F7209528232083D1
:10607000DF91CF911F910F91FF90EF90DF90BF9034
:10608000AF900895DC011C96ED91FC911D97E05CAA
:10609000FF4F2191319180819181281B390B2F7302
:1060A0003070C90108958DEA96E00E944230892B34
:1060B00011F00E94112F0895DC011C96ED91FC91C6
:1060C0001D97E05CFF4F20813181E054F040DF01FB
:1060D000AE5BBF4F8D919C9111972817390719F42A
:1060E0002FEF3FEF07C08D919C91E80FF91F808142
:1060F000282F30E0C9010895DC011C96ED91FC9138
:106100001D97E05CFF4F20813181E054F040DF01BA
:10611000AE5BBF4F8D919C9111972817390719F4E9
:106120002FEF3FEF10C08D919C911197E80FF91F51
:1061300020818D919C91119701968F73907011968B
:106140009C938E9330E0C9010895DC0191968C9167
:106150009197882339F05496ED91FC915597808161
:1061600086FFF9CF91961C920895CF93DF93EC01AF
:10617000EE85FF85E05CFF4F20813181E054F040E7
:106180002F5F3F4F2F733070DF01AE5BBF4F8D919C
:106190009C91119728173907D1F3E05CFF4F80815C
:1061A0009181E054F040E80FF91F6083EE85FF8590
:1061B000E05CFF4F31832083EE89FF89208181E0FD
:1061C00090E00F8C02C0880F991F0A94E2F7282BE9
:1061D000208381E089A3EC89FD89808180648083AC
:1061E00081E090E0DF91CF9108958F929F92AF92DE
:1061F000BF92CF92DF92EF92FF920F931F9300D046
:1062000000D00F92EDB7FEB7319684E0ADB7BEB7C0
:1062100011968C9383E0818387E0828385E083837A
:1062200081E084838DEA96E065E276E049E656E017
:106230002DEC30E00CEC10E0B8ECEB2EF12CA9ECDE
:10624000CA2ED12CFAECAF2EB12CEEEC8E2E912C66
:106250000E94882F0F900F900F900F900F901F911A
:106260000F91FF90EF90DF90CF90BF90AF909F90F5
:106270008F900895CF93DF930E94E02A87ED96E0F8
:106280000E9432320E943529C3E5D0E30E940813F0
:106290002097E1F30E945330F9CFFC0104C08091B4
:1062A000F100819361506623D1F7289884E68093AA
:1062B000D00608959FB7F89487708093E900809185
:1062C000F2009FBF0895282F8091D1068823C1F046
:1062D00057FF1AC015C028989093D0068091F100FE
:1062E0008193E217F307B9F74115510539F0809111
:1062F000F200882319F48BE68093E800AFBF02C058
:106300004FEF5FEFCA010895AFB7F894277020935D
:10631000E9008091F200282F30E0241735070CF4B3
:10632000A901FB019B01240F311D94E6DACFA1E006
:10633000B0E0EDE9F1E30C943636BE016F5F7F4FBC
:1063400041E050E00E946331019719F02FEF3FEFD9
:1063500003C08981282F30E0C9012196E2E00C9426
:1063600052362FB7F89487708093E9008091E80047
:1063700085FD02C090E004C08091F20090E4981B7B
:106380002FBF892F08951092E9001092D306109222
:10639000D2069093D5068093D4060895FF920F936A
:1063A0001F93F82E142F052F4091D4065091D50637
:1063B000212F302FC901DC01FB016EEF29C0F7FE50
:1063C00002C0949101C090812091D2063091D306F1
:1063D00024173507ACF48091E8008570E1F38091D3
:1063E000E80082FF03C02FEF3FEF17C09093F1004A
:1063F000C90101968F739070892B11F46093E800A6
:106400002F5F3F4F3093D3062093D20611973196DA
:106410001097A9F6812F902F9C01C9011F910F9110
:10642000FF9008950F931F939C01162F072F8091C3
:10643000E80082FFFCCFC901612F0E944D318BEF34
:106440008093E800812F902F1F910F9108958093E2
:10645000E9008091F200882319F08AE38093E80034
:10646000089508951092D10681E08093D70080EAC4
:106470008093D80082E189BD09B400FEFDCF61E0C0
:1064800070E080E090E00E94BC2A80E98093D80010
:106490008CE08093E2001092E000559A209A0895D3
:1064A000A0E0B0E0E6E5F2E30C942A36E82E942E64
:1064B000852E8091D106882309F18B01242F352F59
:1064C000C901EC016AEFF62E57E0752E7E208E2D65
:1064D00090E040E2A42EB12CA822B9223AE3632E28
:1064E00020E4C22ED12CC822D9224CC08E2D0E946D
:1064F000B131282F882361F4FA9419F42FEF3FEF7C
:106500004CC061E070E080E090E00E94BC2A3AC09C
:1065100090E0C817D9070CF42C2FC21BD1094FB734
:10652000F8947092E900A114B10421F406C010920D
:10653000F10021502223D9F719C0E7FC03C0F8016C
:10654000922F10C0C801322F06C0FC010196E491C1
:10655000E093F10031503323C1F706C0819180935D
:10656000F10091509923D1F7020F111D8091E8009D
:1065700085FF05C0209729F4C114D10411F0609261
:10658000E8004FBF209709F0B1CF5D9884E6809373
:10659000CF06292D382DC9019C01C901CDB7DEB721
:1065A000EEE00C9446361F920F920FB60F92112414
:1065B0002F933F934F935F936F937F938F939F930B
:1065C000AF93BF93EF93FF938091E1001092E100AE
:1065D000982F93FF0FC01092E90081E08093EB00A9
:1065E0001092EC0082E38093ED001092D10688E0D7
:1065F0008093F00092FF28C083E00E94273282E05F
:106600000E945A31882321F087E196E00E949C2C59
:106610008091CF06882351F08091CF0681508093DE
:10662000CF068091CF06882309F45D9A8091D00629
:10663000882351F08091D00681508093D0068091BC
:10664000D006882309F4289AFF91EF91BF91AF916A
:106650009F918F917F916F915F914F913F912F917A
:106660000F900FBE0F901F901895A1E0B0E0EBE3E4
:10667000F3E30C94343619828E010F5F1F4FC8016B
:106680000E94C22CC8010E94AB35898190E02196FE
:10669000E4E00C9450361F920F920FB60F92112423
:1066A000CF92DF92EF92FF920F932F933F934F93EE
:1066B0005F936F937F938F939F93AF93BF93EF936A
:1066C000FF93DF93CF93CDB7DEB76197DEBFCDBF2A
:1066D0001092E9008091E80083FFEBC0CE010196A3
:1066E00068E00E944D3182EF8093E800998197FF26
:1066F00005C08091E80080FFFCCF03C08EEF80933F
:10670000E800292F30E0C90180769070892B09F0CC
:10671000B1C08A81882329F41092F1001092F1000F
:10672000BDC0813009F4BAC0833009F4B7C08530E8
:1067300049F48091E80080FFFCCF8B8180688093D2
:10674000E300ACC0863009F06BC00C81EF80F884A8
:10675000023071F580E090E00E94C3310E94353331
:1067600099E079E0C72ED12CCC0EDD1EF601292F41
:1067700011922A95E9F799870A8791E09E8790E818
:10678000988B9AEF998B2091D2063091D306275F90
:106790003F4F3C872B878D87C7010E94C33180E024
:1067A000B60149E050E00E94CE310E94353376C0F8
:1067B000C7010E94C331023241F482E290E00E949C
:1067C000A335892B09F46EC069C0013079F48F813B
:1067D0009885089719F481E08093D6068091D606B3
:1067E000882309F063C0E1E4FDE013C0033009F041
:1067F00059C08B81882319F4E3E0FDE00AC08230A0
:1068000019F4E7E0FDE005C0813009F04BC0E9E292
:10681000FDE0449180E8BF0150E00E94CE313EC0CF
:10682000873009F43FC0883021F481E08093F10083
:1068300035C0893099F523703070232B99F5E6E641
:10684000FDE091E031E026E39093E9003093EB0026
:1068500084918093EC002093ED009F5F31969530FA
:1068600099F78EE78093EA001092EA008B8180937B
:10687000D10614C08F8198850E94C3318D818823F1
:1068800029F4CE0101960E94CE2C06C0823051F42C
:10689000CE0101960E947434882321F08EEF8093FC
:1068A000E80007C081E28093EB0003C0E3E5FDE070
:1068B000B0CF6196DEBFCDBFCF91DF91FF91EF9159
:1068C000BF91AF919F918F917F916F915F914F9108
:1068D0003F912F910F91FF90EF90DF90CF900F900D
:1068E0000FBE0F901F901895FC0191818081813A15
:1068F00031F4913089F080E0933089F40DC0813219
:1069000069F49B3021F482818093500305C09A3052
:1069100029F482818093510381E0089580E00895F5
:10692000FC0110820895FC011382128286EB93E031
:10693000918380830895EF92FF920F931F938C01B0
:10694000E62EDC01ED91FC910480F581E02D0995A6
:10695000F82ED801ED91FC910680F781E02DC80159
:106960006E2D09958F2D90E01F910F91FF90EF9064
:10697000089588ED96E00E94903489ED96E00E949B
:1069800093340895A1E0B0E0E8ECF4E30C943236DF
:1069900089838B017A0184E0BE016F5F7F4F41E004
:1069A00050E00E94503284E4B801A7010E945032A6
:1069B0002196E6E00C944E3682E048E050E00E94DA
:1069C000C2340895FC011682178210861186128641
:1069D000138614823496BF010E94DC340895DC01D2
:1069E000683810F0685829C0E62FF0E067FF13C040
:1069F000E058F04081E090E002C0880F991FEA95CE
:106A0000E2F7809514962C911497282314962C93D2
:106A1000149760E012C0E851F24F6491662319F4B4
:106A200020E030E01DC067FF08C014968C911497D9
:106A30008D7F14968C9314976F77FD0190E06623F9
:106A400021F08681861709F416829F5F3196963071
:106A5000B1F7CD011496BD010E94DC3421E030E095
:106A6000C9010895CF93DF93DC01683810F06858AE
:106A700025C0E62FF0E067FF12C0E058F04081E04B
:106A800090E002C0880F991FEA95E2F714962C91C6
:106A90001497282B14962C93149760E00FC0E8519C
:106AA000F24F64916623D9F167FF08C014968C9168
:106AB0001497826014968C9314976F7716968C9126
:106AC00016978617A9F117968C911797861781F15B
:106AD00018968C911897861759F119968C911997D9
:106AE000861731F11A968C911A97861709F11B9621
:106AF0008C911B978617E1F0ED01E0E0F0E09E2F0E
:106B00008E81882321F4EA0FFB1F668306C09F5FF6
:106B100031962196E630F10591F7963049F481E0FF
:106B200090E013969C938E93129720E030E007C07C
:106B3000CD011496BD010E94DC3421E030E0C90192
:106B4000DF91CF91089580E86AE67DE045E650E068
:106B50000E94CE310895FC0180818F5F808380E8A0
:106B60006FEC7DE049E150E00E94CE310895629FD4
:106B7000D001739FF001829FE00DF11D649FE00D35
:106B8000F11D929FF00D839FF00D749FF00D659F96
:106B9000F00D9927729FB00DE11DF91F639FB00D95
:106BA000E11DF91FBD01CF011124089597FB092EA6
:106BB00007260AD077FD04D086D006D000201AF42C
:106BC000709561957F4F0895F6F7909581959F4F49
:106BD0000895A1E21A2EAA1BBB1BFD010DC0AA1F1E
:106BE000BB1FEE1FFF1FA217B307E407F50720F036
:106BF000A21BB30BE40BF50B661F771F881F991FB1
:106C00001A9469F760957095809590959B01AC01F9
:106C1000BD01CF01089597FB092E05260ED057FD23
:106C200004D0D7DF0AD0001C38F450954095309539
:106C300021953F4F4F4F5F4F0895F6F79095809500
:106C4000709561957F4F8F4F9F4F08952F923F9280
:106C50004F925F926F927F928F929F92AF92BF926C
:106C6000CF92DF92EF92FF920F931F93CF93DF9318
:106C7000CDB7DEB7CA1BDB0B0FB6F894DEBF0FBE75
:106C8000CDBF09942A88398848885F846E847D84C2
:106C90008C849B84AA84B984C884DF80EE80FD80C4
:106CA0000C811B81AA81B981CE0FD11D0FB6F8943A
:106CB000DEBF0FBECDBFED010895EE0FFF1F0590A3
:106CC000F491E02D0994AA1BBB1B51E107C0AA1F38
:106CD000BB1FA617B70710F0A61BB70B881F991F7D
:106CE0005A95A9F780959095BC01CD010895911111
:106CF00006C0803219F089508550D0F70895992741
:086D000088270895F894FFCFE5
:106D08004E6F005965730054582074696D656F752E
:106D18007421006D6F64756C65206C6F636B6564BE
:106D28003F00486F70206368616E6E656C200020BC
:106D380040200053004E2F4100386368002C002C7F
:106D4800205B005D20280029004E4F5420454E410D
:106D5800424C45440053656E64696E6720736574E0
:106D680074696E677320746F2052580A00526573F5
:106D7800657474696E672073657474696E677320CF
:106D88006F6E2052580A0041626F72746564206504
:106D9800646974730A00696E76616C69642073654E
:106DA8006C656374696F6E000D0A496E76616C6973
:106DB8006420696E707574202D2064697363617234
:106DC8006465642107007363616E6E6572206D6F80
:106DD80064650053657474696E67732073617665C2
:106DE8006420746F20454550524F4D0A0052657615
:106DF80065727465642073657474696E6773206660
:106E0800726F6D20454550524F4D0A004C6F6164BA
:106E1800656420666163746F727920646566617564
:106E28006C74730A004B657920616E642063686135
:106E38006E6E656C732072616E646F6D697A6564DD
:106E48000A004F70656E4C52536E67205458207379
:106E580074617274696E672000206F6E2048572035
:106E68000050504D0052535349005344410053437E
:106E78004C00525844005458440041494E004C427A
:106E88004545500053504B54524D00534255530002
:106E980053554D44004C4C494E440000342B3400AB
:106EA8003800382B340031320031322B340031367F
:106EB8000001000000C01200001A400AA1204EA5DF
:106EC800001B1E27522C23308025000005400AA1F4
:106ED800204EA50020244EA52C2330004B00000690
:106EE800400AD0009D49007B289D492C233000E1B1
:106EF800000005400A4501D7DC03B81E0EBF002379
:106F08002E48E801008A400A6001555502AD1E204E
:106F1800000023C88025000005400AA1204EA500D6
:106F280020244EA52C23300002000200020002009B
:106F38000200020002000200020002000200020039
:106F480002000200020002FF00E100000000000051
:106F58000101610265026A026E02720276027A0219
:106F68007E0284028B02900295029B029B029B0286
:106F78009B0235019C02A002A202A602A902AE024F
:106F8800350100070B0C10111500160A13223129C0
:106F980000000000732C242D122C392C202C982C46
:106FA8009C2C00000000B530242D42307C305C3031
:106FB800A530000000009B34242D3235EF34E23434
:1070000055C000006EC000006CC000006AC00000E7
:1070100068C0000066C0000064C0000062C00000DC
:1070200060C000005EC00000F2C400005AC0000052
:1070300058C0000056C0000054C0000052C00000FC
:1070400050C0000078C000004CC000004AC00000E2
:1070500048C0000046C0000044C0000042C000001C
:1070600040C000003EC000003CC000003AC000002C
:1070700038C0000036C0000034C0000032C000003C
:1070800030C000002EC000002CC000002AC000004C
:1070900028C0000026C0000024C0000022C000005C
:1070A00020C000001EC000001CC0000011241FBE34
:1070B000CFEFDAE0DEBFCDBF11E0A0E0B1E0E2E368
:1070C000FFE702C005900D92A83AB107D9F711E089
:1070D000A8EAB1E001C01D92AE3BB107E1F78FD342
:1070E00026C78ECFF89410926F00109281001092F4
:1070F00085001092840081E085BF15BE47985D9A97
:10710000289A0C94000008952091B2013091B301A7
:107110002F5F3F4F3093B3012093B201932F37FF7E
:1071200003C08EEF831B982F990F921710F4479886
:107130000895479A08951F920F920FB60F92112447
:107140002F938F939F93EF93FF931092850010924C
:1071500084008091A8019091A901009741F00197C6
:107160009093A9018093A801892B09F45D9A8091DD
:10717000AA019091AB01009741F001979093AB0168
:107180008093AA01892B09F4289AE0E0F0E0859128
:1071900094918F5F9F4F49F08091AC019091AD0128
:1071A00001969093AD018093AC01FF91EF919F9177
:1071B0008F912F910F900FBE0F901F90189584E024
:1071C0008093E9000DC08091E8008B778093E80000
:1071D00003C08EB3882351F08091E80082FFF9CF7D
:1071E0008091E80085FFEFCF8091F1000895982FFE
:1071F00083E08093E9008091E80085FD0DC08091D7
:10720000E8008E778093E80003C08EB3882369F08E
:107210008091E80080FFF9CF9093F1005D9884E6BB
:1072200090E09093A9018093A80108954F925F92F6
:107230006F927F928F929F92AF92BF92CF92DF9286
:10724000EF92FF920F931F93CF93DF9384E080938D
:10725000E9008091E80082FF57C2289884E690E018
:107260009093AB018093AA01AADF182F853481F493
:107270008CE49DE19093AD018093AC0107B600FCD6
:10728000FDCFF999FECF81E180935700E89503C0C7
:10729000843519F494DF8DE00DC28C34E1F3803530
:1072A000D1F3843721F484E4A2DF80E003C2813685
:1072B00011F489E5FFC18134B1F481DF182F7FDF3C
:1072C00090E0880F991FAA2797FDA095BA2F312F1C
:1072D000330F20E0442737FD4095542F822B932B0A
:1072E000A42BB52BB8C1803711F483E5E3C18335F6
:1072F00049F4C0E0D1E089917ADF21E0C730D207BC
:10730000D1F7D9C1863521F481E371DF80E3D2C1A1
:10731000833731F487E86BDF85E969DF8EE1CAC125
:107320008536B9F4E0E0F0E093E085E09093570013
:10733000E89507B600FCFDCF80935700E89507B6A7
:1073400000FCFDCFE058FF4FA0E7E030FA0771F7EF
:10735000A2CF823739F4E1E0F0E089E08093570072
:107360008491A8C1863439F4E0E0F0E089E08093AC
:10737000570084919FC18E3439F4E3E0F0E089E056
:1073800080935700849196C1813539F4E2E0F0E0B2
:1073900089E08093570084918DC1823631F489E56C
:1073A00026DF80E024DF80E885C1823419F087364B
:1073B00009F0E5C01092AD011092AC0100DF082F7A
:1073C000FEDEF82EFCDE682E8554823008F071C196
:1073D000902F80E0CF2DD0E0C82BD92B10926F00DA
:1073E000173609F04BC081E180935700E895DD2402
:1073F000CC24C3943FC0E090AE01F090AF01009167
:10740000B0011091B101B6E46B16D9F4ED2DF0E0A6
:10741000EE29FF29E4918E2FEADEDD2081F082E063
:1074200090E0A0E0B0E0E80EF91E0A1F1B1FE092FA
:10743000AE01F092AF010093B0011093B101DC24D2
:1074400018C0D801C701B695A7959795879559D5C6
:10745000CEDE82E090E0A0E0B0E0E80EF91E0A1F68
:107460001B1FE092AE01F092AF010093B0011093A8
:10747000B1012197209709F0BECF7DC08090AE0169
:107480009090AF01A090B001B090B10196E4691660
:1074900009F05DC083E0F40180935700E89507B6DA
:1074A00000FCFDCF54C0F6E46F1661F5772031F192
:1074B000E090AE01F090AF010091B0011091B101E8
:1074C0007EDED82ECC24852D90E08C299D29F701D5
:1074D0000C0140925700E895112482E090E0A0E072
:1074E000B0E0E80EF91E0A1F1B1FE092AE01F092F9
:1074F000AF010093B0011093B10102C060DE582EBD
:10750000742423C0E090AE01F090AF010091B0016F
:107510001091B10116950795F794E79450DE682F06
:10752000C701F7D48091AE019091AF01A091B00155
:10753000B091B1010296A11DB11D8093AE0190934F
:10754000AF01A093B001B093B101219704C05524BD
:10755000772444244394209709F0A5CF96E4691634
:1075600041F485E0F40180935700E89507B600FCEC
:10757000FDCF8DE03CDE82E080936F009CC08334C1
:1075800071F40091AE011091AF0119DE90E021E09D
:10759000F8010C0120935700E89511247CCE833626
:1075A00019F5E090AE01F090AF010091B00110919B
:1075B000B10105DEF701E16090E021E00C012093CC
:1075C0005700E895112482E090E0A0E0B0E0E80EDA
:1075D000F91E0A1F1B1FE092AE01F092AF0100934B
:1075E000B0011093B10157CE8D3661F4E091AE0138
:1075F000F091AF0185E080935700E89507B600FC55
:10760000FDCF49CE823551F4E091AE01F091AF014A
:1076100005911491812FEBDD802F4CC0843421F52E
:10762000E090AE01F090AF010091B0011091B10176
:1076300016950795F794E794C2DD682FC70169D4C2
:107640008091AE019091AF01A091B001B091B101D4
:107650000296A11DB11D8093AE019093AF01A0933E
:10766000B001B093B10117CE843609F5E090AE01B8
:10767000F090AF010091B0011091B101D801C701A4
:10768000B695A795979587953CD4B1DD82E090E0BB
:10769000A0E0B0E0E80EF91E0A1F1B1FE092AE0149
:1076A000F092AF010093B0011093B10104C08B318F
:1076B00011F08FE39CDD83E08093E9009091E80076
:1076C0008091E8008E778093E80095FF04C010C099
:1076D0008EB38823C9F08091E80080FFF9CF8091B4
:1076E000E8008E778093E80003C08EB3882361F0B2
:1076F0008091E80080FFF9CF84E08093E9008091D9
:10770000E8008B778093E800DF91CF911F910F9174
:10771000FF90EF90DF90CF90BF90AF909F908F90B1
:107720007F906F905F904F9008959091B601892F50
:107730008F77813249F58091B7018032A1F0813293
:1077400019F5913A09F58091E800877F8093E80068
:107750008DE091E067E070E00BD28091E8008B77DC
:107760008093E8000895913279F48091E800877F52
:107770008093E8008DE091E067E070E05DD2809159
:10778000E8008E778093E800089582E061EC42E0A3
:10779000B5D083E061E842E1B1D084E060E842E145
:1077A000ADC084B7877F84BF88E10FB6F89480931B
:1077B0006000109260000FBE20E880E090E00FB6FD
:1077C000F89420936100809361000FBE81E085BF33
:1077D00092E095BF3F9A209A559AE1E6F0E0208327
:1077E000108247985D9A289A109289008AEF8093B8
:1077F000880090936F0083E080938100F0C04091F7
:10780000000850910108109201081092000894B7E6
:1078100014BE88E10FB6F894809360001092600067
:107820000FBE292F30E0F901E270F07091FD18C011
:1078300090FF05C0859194918F5F9F4F81F423FF46
:107840000FC08091090190910A014817590741F032
:10785000E0E0F0E0859194918F5F9F4F09F042DC6A
:10786000A0DF78941092AD011092AC010CC0DEDC68
:1078700036D38091AC019091AD0181549F4110F0BD
:107880001092140141DC80911401882381F78091CA
:10789000E00081608093E00025DC80E090E00895C6
:1078A000FA01923049F0933061F09130F9F485E1BA
:1078B00091E022E130E01EC087E291E02EE330E06B
:1078C00019C0882329F485E691E024E030E012C055
:1078D000813029F489E691E022E230E00BC0823069
:1078E00029F48DE891E028E130E004C080E090E0E8
:1078F00020E030E091838083C90108958093E900FE
:107900008091EB0081608093EB001092ED0060931A
:10791000EC004093ED008091EE00881F8827881FBF
:1079200008958091B60188238CF403C08EB3882318
:10793000B1F08091E80082FFF9CF8091E8008B7769
:107940008093E80008958EB3882349F08091E80081
:1079500080FFF9CF8091E8008E778093E80008954A
:10796000EF92FF920F931F9345D04CD008ED10E09B
:10797000F80180818F778083808180688083808117
:107980008F7D808319BC1EBA1092B40180EEE82E60
:10799000F12CF70180818B7F8083F80180818160E9
:1079A000808380E060E042E0A9DFE1EEF0E08081EA
:1079B0008E7F8083E2EEF0E0808181608083808131
:1079C00088608083F70180818E7F8083F8018081C9
:1079D000806180831F910F91FF90EF900895E7EDF4
:1079E000F0E08081816080838AE482BF81E08093BF
:1079F000B501B6CFE8EDF0E080818E7F80831092F4
:107A0000E20008951092DA001092E10008951F92AA
:107A10000F920FB60F9211242F933F934F935F93C2
:107A20006F937F938F939F93AF93BF93EF93FF9346
:107A30008091DA0080FF1BC08091D80080FF17C0C2
:107A40008091DA008E7F8093DA008091D90080FFE8
:107A50000BC080E189BD82E189BD09B400FEFDCF84
:107A600081E08EBB3BD203C019BC1EBA37D28091D5
:107A7000E10080FF17C08091E20080FF13C0809179
:107A8000E2008E7F8093E2008091E200806180932B
:107A9000E2008091D80080628093D80019BC85E014
:107AA0008EBB1CD28091E10084FF2CC08091E2004B
:107AB00084FF28C080E189BD82E189BD09B400FE50
:107AC000FDCF8091D8008F7D8093D8008091E10018
:107AD0008F7E8093E1008091E2008F7E8093E200B0
:107AE0008091E20081608093E2008091B40188235C
:107AF00031F48091E30087FD02C081E001C084E0A1
:107B00008EBBECD18091E10083FF21C08091E20027
:107B100083FF1DC08091E100877F8093E10082E0B8
:107B20008EBB1092B4018091E1008E7F8093E100C2
:107B30008091E2008E7F8093E2008091E20080617C
:107B40008093E20080E060E042E0D8DEC7D1FF91A0
:107B5000EF91BF91AF919F918F917F916F915F91C5
:107B60004F913F912F910F900FBE0F901F9018953E
:107B70009C014091BC015091BD014617570718F474
:107B8000F90190E044C06115710511F0AB01F8CF27
:107B90008091E8008E778093E80040E050E0F0CFDD
:107BA0008EB3882309F444C0853009F443C0809122
:107BB000E80083FF02C081E008958091E80082FD23
:107BC00031C08091E80080FF22C08091F300909145
:107BD000F200782F60E0292F30E0262B372B07C0EA
:107BE00081918093F100415050402F5F3F4F4115EC
:107BF000510519F02830310598F390E0283031050F
:107C000009F491E08091E8008E778093E8004115B7
:107C1000510531F6992321F605C08EB3882341F032
:107C2000853041F08091E80082FFF7CF80E0089531
:107C300082E0089583E008959C016115710529F49F
:107C40008091E8008B778093E800F90126C08EB31D
:107C5000882391F1853091F18091E80083FF02C083
:107C600081E008958091E80082FFF1CF06C0809105
:107C7000F10081936150704059F02091F3008091A0
:107C8000F200322F20E090E0822B932B892B79F7A2
:107C90008091E8008B778093E80061157105B9F653
:107CA00005C08EB3882341F0853041F08091E80013
:107CB00080FFF7CF80E0089582E0089583E0089583
:107CC0000F931F93DF93CF9300D0CDB7DEB7E6EBD2
:107CD000F1E08091F100819381E0EE3BF807C9F774
:107CE00024DD8091E80083FFE4C08091B60190918B
:107CF000B701953009F46DC0963040F4913081F1B0
:107D0000913070F0933009F0D4C02AC0983009F453
:107D1000A3C0993009F4B2C0963009F0CAC07CC043
:107D2000803809F4C6C0823809F0C3C08091BA0116
:107D300087708093E9008091EB001092E900209118
:107D4000E800277F2093E80090E025E0969587954E
:107D50002A95E1F781708093F1001092F10087C0BD
:107D6000882319F0823009F0A4C08F71823009F0A5
:107D7000A0C08091B801882331F52091BA01277005
:107D800009F497C02093E9008091EB0080FF1BC0AD
:107D9000933021F48091EB00806213C08091EB005E
:107DA00080618093EB0081E090E002C0880F991F12
:107DB0002A95E2F78093EA001092EA008091EB00A6
:107DC00088608093EB001092E9008091E800877F43
:107DD00051C0882309F06DC01091B8011F770FB70B
:107DE000F8948091E800877F8093E8009ADD809185
:107DF000E80080FFFCCF8091E3008078812B8093A6
:107E0000E30080688093E300112311F482E001C055
:107E100083E08EBB0FBF4DC08058823008F049C050
:107E20008091B8019091B9016091BA01AE014F5FA4
:107E30005F4F36DDBC01009709F43BC08091E8003C
:107E4000877F8093E80089819A8192DE8091E800A3
:107E50008B778093E8002DC0803859F58091E80039
:107E6000877F8093E8008091B4018093F100809136
:107E7000E8008E778093E80054DD1BC08823C9F4A6
:107E80009091B8019230A8F48091E800877F8093A8
:107E9000E8009093B40145DD8091B401882331F46A
:107EA0008091E30087FD02C081E001C084E08EBBC9
:107EB0006CDC8091E80083FF0AC08091EB00806257
:107EC0008093EB008091E800877F8093E8000F901B
:107ED0000F90CF91DF911F910F91089508951F93F7
:107EE0008EB3882361F01091E9001092E90080912F
:107EF000E80083FF01C0E4DE17701093E9001F91D2
:107F00000895F999FECF92BD81BDF89A992780B561
:107F10000895262FF999FECF1FBA92BD81BD20BDCD
:107F20000FB6F894FA9AF99A0FBE01960895F8944C
:107F3000FFCF4341544552494E4100777700080036
:107F400000000000000801120110010200000841B9
:107F500023360001000201000109023E0002010077
:107F60008032090400000102020100052400100112
:107F7000042402040524060001070582030800FF0B
:107F800009040100020A00000007050402100001B4
:107F90000705830210000104030904220341007253
:107FA000006400750069006E006F0020004C0065E1
:107FB000006F006E006100720064006F0000001826
:107FC00003410072006400750069006E006F0020BC
:0A7FD000004C004C004300000000CC
:00000001FF
